:020000040800F2
:10000000008001209D400008ED400008ED40000800
:10001000ED400008ED400008ED4000080000000041
:10002000000000000000000000000000ED4000089B
:10003000ED40000800000000ED4000089D1F000892
:10004000ED400008ED400008ED400008ED400008DC
:10005000ED400008ED400008ED400008ED400008CC
:10006000ED400008ED400008ED400008ED400008BC
:10007000ED400008ED400008ED400008ED400008AC
:10008000ED400008ED400008ED400008ED4000089C
:10009000ED400008ED400008ED400008ED4000088C
:1000A000ED400008ED400008ED400008ED4000087C
:1000B000ED400008ED400008ED400008ED4000086C
:1000C000ED400008ED400008ED400008ED4000085C
:1000D000ED40000835200008ED400008DD20000854
:1000E000ED400008ED400008ED400008ED4000083C
:1000F000ED400008ED400008ED400008ED4000082C
:10010000ED400008ED400008ED400008ED4000081B
:100110002D22000885210008ED400008ED40000870
:10012000ED400008ED400008ED400008ED400008FB
:10013000ED400008ED400008ED400008ED400008EB
:10014000ED400008ED400008ED4000082D47000894
:10015000ED400008ED400008ED400008ED400008CB
:10016000ED400008ED400008ED400008ED400008BB
:10017000ED400008ED400008ED40000800000000E0
:08018000ED400008ED4000080D
:1001880010B5054C237833B9044B13B10448AFF3C9
:1001980000800123237010BD6404002000000000CB
:1001A800C48B0008084B10B51BB108490848AFF3C9
:1001B80000800848036803B910BD074B002BFBD02B
:1001C800BDE81040184700BF000000006804002088
:1001D800C48B0008640400200000000070B50F4EB6
:1001E8000F4D761BB61018BF002405D0013455F802
:1001F800043B9847A642F9D10A4E0B4D761B08F0EE
:10020800DDFCB61018BF002406D0013455F8043BB5
:100218009847A642F9D170BD70BD00BFC8930008C9
:10022800C8930008D0930008C8930008024B13B184
:10023800024800F005B870470000000055020008A9
:10024800002301461A46184600F014B838B5074D81
:10025800074C2C1BA41005D0013C55F8043D9847C9
:10026800002CF9D1BDE8384008F0AEBCD4930008A2
:10027800D09300082DE9F047254C2568D5F848416A
:100288000646884692469946C4B360681F2817DC1C
:10029800431C76B104EB80050122C5F888A0D4F888
:1002A800881182401143022EC4F88811C5F80891BC
:1002B8001ED00230636044F820800020BDE8F0873B
:1002C800144B03B34FF4C870AFF300800446D0B1A9
:1002D800D5F84831002780E88800C5F848413846F5
:1002E8000123C4F88871C4F88C71002EE1D0D1E7DD
:1002F800D4F88C110A43C4F88C21DAE705F5A67402
:10030800C5F84841C1E74FF0FF30BDE8F08700BFAE
:10031800848D00080000000080B483B000AF03465D
:10032800FB71094997F907305B09FA7902F01F0256
:10033800012000FA02F241F8232000BF0C37BD4625
:100348005DF8047B704700BF00E100E080B483B033
:1003580000AF03463960FB7197F90730002B0BDAC1
:100368000D49FB7903F00F03043B3A68D2B212013E
:10037800D2B20B441A7609E0084997F907303A686F
:10038800D2B21201D2B20B4483F8002300BF0C375B
:10039800BD465DF8047B704700ED00E000E100E039
:1003A80080B582B000AF78607B68013BB3F1807F95
:1003B80001D301230FE00A4A7B68013B53600F21F8
:1003C8004FF0FF30FFF7C2FF054B00229A60044B45
:1003D80007221A60002318460837BD4680BD00BFB3
:1003E80010E000E080B582B000AF9F4A9E4B5B6989
:1003F80043F4007353619C4B9C4ADA6000F092F915
:100408009B4A9B4BDB6C43F00103D364984A984B9F
:10041800DB6C43F00203D364954A954BDB6C43F0E5
:100428000403D364924A924BDB6C43F00803D36411
:100438004FF090424FF090431B6803F070531360E5
:100448008C4B00221A608C4B00221A608A4A8A4B15
:100458001B6843F480331360874A874B1B6843F05B
:1004680050031360844B0C229A61844B1B68844AA6
:10047800A2FB03239B091846FFF792FF814B142226
:100488001A80814B00221A80804B00221A80804BF0
:1004980000221A807F4B00221A8002F0D7FB7E4B85
:1004A80045F255521A607C4B4FF6FF729A60022053
:1004B80000F0CEF9784B02225A60022000F0C8F909
:1004C800754B4CF6CC421A606B4A6B4BDB6843F0B9
:1004D8000503D360684A684BDB6823F00A03D360DE
:1004E800022000F0B5F900F08DFB634B1B699BB24D
:1004F80003F003039BB2DB439BB203F003039AB2FE
:10050800664B1A80654B1B88002B03D1644B002275
:100518001A7022E0634B5B6B03F00F03002B08D1CA
:100528005E4B1B88DBB243F02003DAB25C4B1A70D7
:1005380013E05C4B5B6B03F00F03012B08D1574BA7
:100548001B88DBB243F01003DAB2554B1A7004E093
:10055800524B1B88DAB2524B1A70514B1B7803F07E
:100568000303DAB2504B1A704D4B1B780F2B03D88C
:100578004E4B00221A7002E04C4B01221A7000F018
:1005880077FD00F07BFE00F05FFF01F05DF8484B5F
:1005980000221A7003F062FE322000F059F907F0C9
:1005A8009FFF642000F054F907F028FC642000F055
:1005B8004FF93B4B1B78022B02D107F09DFD08E059
:1005C800374B1B781F2B02D807F064FC01E007F0BB
:1005D800FBFC334B1B78102B01D902F037FB64204E
:1005E80000F036F92B4B41F288321A8007E02A4B8B
:1005F8004AF6AA221A602E4B1B78002B04D1254BF1
:100608001B88002BF3D100E000BF294B1B78002B7F
:1006180002D1284801F0C0F9214B1B780F2B04D9CF
:1006280007F06EFE01F052FEF6E71D4B1B78002B1B
:1006380003D01B4B1B78032B0FD103F09DF901F05E
:10064800E9FB0346FB80FB88002B60D0FB887B71AD
:100658007B79184605F042FC59E0114B1B78012BB9
:100668002AD107F04DFE2DE000ED00E00007FA0565
:10067800001002400004004800080048540400200C
:10068800D34D6210B0B40020CE1A0020D21A002038
:10069800CC1A0020785C0020003000402C5D00203F
:1006A800D01A0020D45C00206C380120824E012032
:1006B8007738012048040020154B1B78022B01D104
:1006C80007F066FE134B1A68134B1B689A4211D049
:1006D800104B1B685A1C0F490A601B78184601F01A
:1006E80021F90C4B1A680D4B1B689A4202D3094B2F
:1006F8000B4A1A6001F08EFB0346FB80FB88002B37
:100708008AD0FB887B717B79184607F059FD83E70F
:10071800D01A0020E0040020DC040020600400203F
:100728007870012080B400AF444A444B9B6D43F07D
:100738008053936500BF424B5B6903F48063002BD1
:10074800F9D13F4A3E4B1B6823F4806313603C4A4F
:100758003B4B1B6843F44073136000BF384B5B6925
:1007680003F48063002BF9D1364A364B1B6843F4F7
:1007780081731360314A314B1B6823F08073136017
:1007880000BF2E4B1B6803F00073002BF9D12B4AD6
:100798002A4BD3F8903023F03D03C2F89030274A13
:1007A800264BD3F8903043F01803C2F89030234A10
:1007B800224BD3F8903043F00103C2F8903000BFC9
:1007C8001E4BD3F8903003F00203002BF8D000BF83
:1007D8001A4B1B6803F00203002BF9D0174A174B7A
:1007E8001B6823F0F0031360144A144B1B6843F092
:1007F800B0031360114A114B1B6843F00D031360DB
:1008080000BF0E4B1B6803F00203002BF9D00B4A04
:100818000A4B9B6843F410539360084A074BD3F87C
:10082800883043F04063C2F88830074B074A1A60A3
:1008380000BFBD465DF8047B704700BF0010024052
:10084800007000400020024054040020006CDC02CC
:1008580080B483B000AF0346FB80094AFB8813804D
:1008680003E0084B4AF6AA221A60054B1B88002BA6
:10087800F7D100BF0C37BD465DF8047B704700BF59
:10088800CC1A00200030004080B582B000AFA7230A
:100898007B6004E000F00AF87B68013B7B607B68C2
:1008A800002BF7D100BF0837BD4680BD80B483B0A8
:1008B80000AF0A4B1B680A4AA2FB0323DB0C7B60D0
:1008C80002E07B68013B7B607B68002BF9D100BFAD
:1008D8000C37BD465DF8047B704700BF5404002008
:1008E80083DE1B4380B500AF514B1B78012B40D1F1
:1008F800504B1B6903F48043002B3AD1012102209D
:1009080007F078FF03461A464B4B1A704A4B1B7880
:1009180003F00803002B02D007F0EEFB29E0464B5A
:100928001B7803F01503002B10D0FF2201210220B1
:1009380007F09CFE404B1B7803F00103002B18D0F6
:100948003E4B9B6C9AB23E4B1A8012E03A4B1B7896
:1009580003F00203002B0CD00121032007F04AFF0B
:1009680003461A46344B1A70354B00221A8007F09A
:10097800C3FB344B1B88002B57D1324B14221A80EF
:10098800314B4AF6AA221A60304B1B88002B02D141
:100998002F4B04229A612F4B1B88002B02D12C4B22
:1009A80008229A612C4B1B780133DAB22A4B1A7051
:1009B800294B1B78312B38D9274B00221A7000F0AD
:1009C8004DF81F4B1B88002B2FD01D4B1B88013B5C
:1009D8009AB21B4B1A801A4B1B88052B1BD1144B40
:1009E8001B78012B17D1202007F0EAFB452007F0E0
:1009F800E7FB582007F0E4FB352007F0E1FB732004
:100A080007F0DEFB212007F0DBFB202007F0D8FBF6
:100A18000B4B05221A800A4B1B88002B05D1044B6F
:100A28001B78012B01D107F0A5FB00BF80BD00BFDB
:100A38007670012000040048C0040020D45C002027
:100A480074700120B0B4002000300040CE1A00209D
:100A580000080048D21A0020C104002080B582B0E6
:100A680000AF5E4B1B699BB203F003039BB2DB43F1
:100A78009BB203F00303FB80594B1B88FA889A4208
:100A880000F0A780574B1B787B71554AFB88138071
:100A9800534B1B88002B03D1524B00221A7022E0C3
:100AA800514B5B6B03F00F03002B08D14C4B1B8899
:100AB800DBB243F02003DAB24A4B1A7013E04A4B18
:100AC8005B6B03F00F03012B08D1454B1B88DBB28E
:100AD80043F01003DAB2434B1A7004E0404B1B8812
:100AE800DAB2404B1A703F4B1B7803F00303DAB2BB
:100AF8003E4B1A707B790F2B03D83A4B1B780F2B80
:100B080006D87B790F2B24D9364B1B780F2B20D88E
:100B180003F054FB314B4FF440229A61344B4AF6B0
:100B2800AA221A604FF4FA70FFF792FE2D4B1B7839
:100B38000F2B03D82F4B00221A7002E02D4B0122F5
:100B48001A702B4B4AF6AA221A6003F087FB00F0B2
:100B58007BFD10220121012007F088FD214B1B7825
:100B6800022B02D107F0C8FA08E01E4B1B781F2B96
:100B780002D807F08FF901E007F026FA194B1B7825
:100B8800102B01D902F062F8194B4AF6AA221A6012
:100B98004FF4FA70FFF75CFE174B41F288321A8067
:100BA80007E0134B4AF6AA221A60144B1B78002B55
:100BB80004D1114B1B88002BF3D100E000BF0F4B71
:100BC8001B78002B02D10E4800F0E6FE034B0C22E6
:100BD8009A6100BF0837BD4680BD00BF00080048C5
:100BE8002C5D0020D01A0020D45C00206C38012035
:100BF80000300040824E0120785C002077380120C8
:100C08004804002080B584B000AF5E4BBB605E4BEB
:100C18007B600023FB730DE0BB681B68DA437B68CD
:100C28001A607B6804337B60BB680433BB60FB7B62
:100C38000133FB73FB7B142BEED9534B1B68002B42
:100C480003D1514B40F283421A604F4B5B68002B33
:100C580003D14D4B45F240725A604B4B9B68002BB9
:100C680002D1494B50229A60474BDB68002B02D1D6
:100C7800454B464ADA60444B1B69002B02D1424B74
:100C8800434A1A61404B5B69002B02D13E4B414AF3
:100C98005A613D4B9B69002B03D13B4B6FF0FF0220
:100CA8009A61394B9B6A002B02D1374B3A4A9A62B8
:100CB800354BDB6A002B03D1334B45F2A852DA627D
:100CC800314B1B6B002B03D12F4B45F2A8521A63F3
:100CD8002D4BDB69002B0AD12B4B5A692A4B9B6998
:100CE8001A40294B9B69DB431343274AD361264BA0
:100CF8001B6A002B03D1244B4FF4FA521A62224B81
:100D08005B6A002B03D1204B4FF4FA525A621E4BF8
:100D18005B6C002B02D11C4B17225A641A4B9B6B3D
:100D2800002B03D1184B4FF0FF329A63164BDB6B45
:100D3800002B03D1144B4FF0FF32DA63124B1B6CBC
:100D4800002B03D1104B4FF0FF321A640E4B9B6CF3
:100D5800002B03D10C4B4FF496729A640A4BDB6C50
:100D6800002B02D1084B0B22DA64074B1B6D002BBA
:100D780002D1054B1F221A6500F010F800BF10378A
:100D8800BD4680BD00C000087C5C0020FB8F92C27D
:100D98000000A8C0F000A8C0250000E180B485B01C
:100DA80000AF2C4BBB602C4B7B600023FB730BE02C
:100DB8007B681A1D7A601A68BB681A60BB680433BE
:100DC800BB60FB7B0133FB73FB7B142BF0D9234BFC
:100DD80000221A70224B00221A70224B00221A702D
:100DE800214B00221A70214B00221A70194B5B6BA1
:100DF80003F0F003002B02D0184BFF221A70154B9A
:100E08005B6B03F47063002B02D0154BFF221A7042
:100E1800104B5B6B03F48053002B02D0124BFF2264
:100E28001A700C4B5B6B03F40053002B02D00F4B72
:100E3800FF221A70074B5B6B03F48043002B02D030
:100E4800084BFF221A7000BF1437BD465DF8047BBB
:100E5800704700BFD45C00207C5C0020A1E000202B
:100E68006A3801209DE000204238012059220120E3
:100E780090B58BB000AF764B3C460FCB07C42380B0
:100E880002341B0C237000BF724B1B6903F48033C0
:100E9800002BF9D16F4B5B69002B05DA6D4B6E4A5D
:100EA8009A606C4B6D4A9A6000BF6A4B1B6903F4E9
:100EB8008033002BF9D1674B694A5A61654A654B03
:100EC8005B6943F48033536100BF624B1B6903F4D1
:100ED8008033002BF9D15F4B1B6903F00103002B12
:100EE80006D05C4A5B4B1B6943F0010313610AE0BF
:100EF800584B1B69184600F0F3FD3F2000F012FD27
:100F08003F2000F00FFD534A524B5B6923F0020368
:100F18005361544B3B62544BBB61544BFB614D4A8C
:100F28004C4B5B6943F001035361002387F827307A
:100F38004CE0BB691A68FB691A60BB691B68DA4335
:100F48003B6A1A60FB690433FB61BB690433BB610C
:100F58003B6A04333B62BB691A68FB691A60BB6968
:100F68001B68DA433B6A1A60FB690433FB61BB699F
:100F78000433BB613B6A04333B6200BF354B1B69DA
:100F880003F48033002BF9D1324B1B6903F00103C2
:100F9800002B06D02F4A2F4B1B6943F00103136126
:100FA8000FE097F82730184600F00CFD294B1B6915
:100FB800184600F095FD212000F0B4FC212000F037
:100FC800B1FC97F82730013387F8273097F8273096
:100FD8000A2BAED91F4A1F4B5B6923F001035361EB
:100FE8001C4A1C4B5B6943F0004353610A20FFF71E
:100FF8002FFC1C4B3B621C4BBB61002387F827303E
:101008001CE03B6A1A1D3A621B68DB437B61BB69C3
:101018001A1DBA611B683B613A697B699A4208D01C
:101028003B46184600F0B8FC0D2000F07BFC00237E
:1010380009E097F82730013387F8273097F82730E9
:10104800142BDED9012318462C37BD4690BD00BFAE
:10105800DC8B00080020024023016745AB89EFCDF7
:10106800C200000100C000087C5C0020D45C0020A5
:1010780080B500AF2D4A2D4B1B6E43F48043136699
:101088004FF090424FF090431B6823F48013136095
:101098004FF090424FF090431B6843F400131360E5
:1010A800234A234B1B6823F480531360204A204BA8
:1010B8001B6843F4005313604FF090424FF0904385
:1010C8005B6A23F4706353624FF090424FF0904391
:1010D8005B6A43F4E0635362154A154B1B6A23F0BD
:1010E80070631362124A124B1B6A43F0E063136287
:1010F800104B114A1A60114B0F4A1A60104B114AD3
:101108001A60114B0F4A1A60104B4FF44072DA60A4
:101118000E4B00225A600D4B00229A600B4B2D2279
:101128001A602520FFF7F8F800BF80BD00100240C4
:10113800000400488004002010730020840400206C
:1011480088040020EC0400208C04002000380140B2
:1011580080B483B000AF0346FB710E4B1B685A1C6A
:101168000C490A60FA791A700A4B1A680A4B1B680C
:101178009A4202D1074B094A1A60094A084B1B6870
:1011880043F08003136000BF0C37BD465DF8047B55
:10119800704700BF880400202C040020EC040020C5
:1011A8000038014080B582B000AFFFF79BFB2A4BA7
:1011B8001A682A4B1B689A4248D0274B1B685A1C4E
:1011C80025490A601B789BB26FEA43436FEA534391
:1011D800FB80214B1A68224B1B689A4202D11E4B96
:1011E800204A1A60FB8848F2F802934205D11E4B48
:1011F8001B78002B01D0002329E0FB8848F2FE026F
:10120800934205D1194B1B78002B01D000231EE017
:10121800FB8848F2F602934205D1154B1B78002B48
:1012280001D0002313E0FB8848F2F80293420BD068
:10123800FB8848F2FE02934206D00E4B4FF4002280
:101248009A610D4BC8221A80FB8800E000231846DB
:101258000837BD4680BD00BF8404002080040020FC
:101268002804002010730020423801205922012050
:101278009DE0002000080048D21A002080B500AF89
:101288001D4A1D4B9B6D43F4802393651B4A1B4BE2
:101298001B6823F470031360184A184B1B6843F447
:1012A80020031360154A154B5B6A23F47F4353628E
:1012B800124A124B5B6A43F4EE435362104B114AD5
:1012C8001A60114B0F4A1A60104B114A1A60114BE1
:1012D8000F4A1A60104B4FF44072DA600E4B00222E
:1012E8005A600D4B00229A600B4B2D221A60272062
:1012F800FFF712F800BF80BD001002400008004848
:1013080090040020F0880020940400209804002015
:10131800984600209C0400200048004080B483B018
:1013280000AF0346FB710E4B1B685A1C0C490A6040
:10133800FA791A700A4B1A680A4B1B689A4202D14A
:10134800074B094A1A60094A084B1B6843F0800397
:10135800136000BF0C37BD465DF8047B704700BFC3
:1013680098040020340400209846002000480040DB
:1013780080B582B000AFFFF7B5FA2A4B1A682A4B3E
:101388001B689A4248D0274B1B685A1C25490A609B
:101398001B789BB26FEA43436FEA5343FB80214BB0
:1013A8001A68224B1B689A4202D11E4B204A1A60C7
:1013B800FB8848F2F802934205D11E4B1B78002B9C
:1013C80001D0002329E0FB8848F2FE02934205D1B0
:1013D800194B1B78002B01D000231EE0FB8848F234
:1013E800F602934205D1154B1B78002B01D0002340
:1013F80013E0FB8848F2F80293420BD0FB8848F2CE
:10140800FE02934206D00E4B4FF400229A610D4B18
:10141800C8221A80FB8800E0002318460837BD461A
:1014280080BD00BF940400209004002030040020F8
:10143800F088002042380120592201209DE0002038
:1014480000080048D21A002080B500AF294A294B6D
:101458009B6D43F480139365274A274B1B6823F041
:1014680040731360244A244B1B6843F000731360D5
:10147800224A224B1B6823F0300313601F4A1F4B7C
:101488001B6843F0200313601B4A1B4B5B6A23F461
:1014980070235362184A184B5B6A43F40023536263
:1014A800164A164B1B6A23F470631362134A134BD4
:1014B8001B6A43F400631362114B124A1A60124B01
:1014C800104A1A60114B124A1A60124B104A1A60DD
:1014D800114B4FF44072DA600F4B00225A600E4BEA
:1014E80000229A600C4B2D221A603520FEF714FF5B
:1014F80000BF80BD0010024000080048000C0048F2
:10150800B0040020B8300020B4040020B804002043
:10151800D09E0020BC0400200050004080B483B05E
:1015280000AF0346FB710E4B1B685A1C0C490A603E
:10153800FA791A700A4B1A680A4B1B689A4202D148
:10154800074B094A1A60094A084B1B6843F0800395
:10155800136000BF0C37BD465DF8047B704700BFC1
:10156800B804002044040020D09E00200050004011
:1015780080B582B000AFFFF7B5F92A4B1A682A4B3D
:101588001B689A4248D0274B1B685A1C25490A6099
:101598001B789BB26FEA43436FEA5343FB80214BAE
:1015A8001A68224B1B689A4202D11E4B204A1A60C5
:1015B800FB8848F2F802934205D11E4B1B78002B9A
:1015C80001D0002329E0FB8848F2FE02934205D1AE
:1015D800194B1B78002B01D000231EE0FB8848F232
:1015E800F602934205D1154B1B78002B01D000233E
:1015F80013E0FB8848F2F80293420BD0FB8848F2CC
:10160800FE02934206D00E4B4FF400229A610D4B16
:10161800C8221A80FB8800E0002318460837BD4618
:1016280080BD00BFB4040020B004002040040020A6
:10163800B830002042380120592201209DE00020C6
:1016480000080048D21A002080B582B000AF5A4A7C
:10165800594B9B6D43F4002393654FF090424FF034
:1016680090431B6823F00F0313604FF090424FF034
:1016780090431B6843F00A0313604FF090424FF009
:1016880090431B6A23F0FF0313624FF090424FF020
:1016980090431B6A43F088031362484B484A1A6018
:1016A800484B474A1A60484B484A1A60484B474AD1
:1016B8001A60484B1B78002B02D1D023FB8067E0CF
:1016C800444B1B780F2B31D8434BDB6C1F2B17D0A7
:1016D8001F2B06D8132B0FD0172B20D00B2B1BD06A
:1016E80020E0392B14D0602B02D0262B0CD019E027
:1016F8004FF41C63FB804BE04FF49C63FB8047E096
:101708004FF44073FB8043E04FF41C73FB803FE0D1
:101718004FF4D073FB803BE0D023FB8038E0682394
:10172800FB8035E0D023FB8000BF31E02A4B1B6DE6
:101738001F2B17D01F2B06D8132B0FD0172B20D0F9
:101748000B2B1BD020E0392B14D0602B02D0262B7A
:101758000CD019E04FF41C63FB8019E04FF49C6334
:10176800FB8015E04FF44073FB8011E04FF41C73CD
:10177800FB800DE04FF4D073FB8009E0D023FB80A1
:1017880006E06823FB8003E04FF44073FB8000BF52
:10179800124AFB88D360114B00225A600F4B00227B
:1017A8009A600E4B2D221A603420FEF7B5FD00BF5B
:1017B8000837BD4680BD00BF00100240A0040020CD
:1017C800305D0020A4040020A8040020D41A0020C2
:1017D800AC040020D01A0020D45C0020004C00404B
:1017E80080B483B000AF0346FB710E4B1B685A1CD4
:1017F8000C490A60FA791A700A4B1A680A4B1B6876
:101808009A4202D1074B094A1A60094A084B1B68D9
:1018180043F08003136000BF0C37BD465DF8047BBE
:10182800704700BFA80400203C040020D41A002000
:10183800004C004080B582B000AFFFF753F82E4B44
:101848001A682E4B1B689A4251D02B4B1B685A1CA6
:1018580029490A601B789BB26FEA43436FEA5343F6
:10186800FB80254B1A68264B1B689A4202D1224BF3
:10187800244A1A60244B1B78102B20D9FB8848F285
:10188800F802934205D1214B1B78002B01D000238D
:101898002EE0FB8848F2FE02934205D11C4B1B78D0
:1018A800002B01D0002323E0FB8848F2F602934284
:1018B80005D1184B1B78002B01D0002318E0164BDC
:1018C800DB68B3F5407F09D1FB8848F2F802934200
:1018D8000BD0FB8848F2FE02934206D00F4B4FF420
:1018E80000229A610E4BC8221A80FB8800E0002370
:1018F80018460837BD4680BDA4040020A004002077
:1019080038040020305D0020D01A00204238012021
:10191800592201209DE00020004C004000080048AA
:10192800D21A002080B582B000AF0346FB71FB7964
:101938001846FFF755FF0A4B1B78002B0BD1094BB4
:101948001B78002B07D1084B1B78002B03D0FB79A1
:10195800184603F043FF00BF0837BD4680BD00BFEF
:10196800D01A0020824E01207738012080B584B03B
:1019780000AF0346FB71FB793033FB73FB7B392BDC
:1019880002D9FB7B0733FB73FB7B1846FFF7CAFFC3
:1019980000BF1037BD4680BD80B584B000AF786009
:1019A80003E0FB7B1846FFF7BDFF7B685A1C7A6093
:1019B8001B78FB73FB7B002BF3D100BF1037BD46B0
:1019C80080BD00BF80B584B000AF0346FB71FB79D2
:1019D8001B09FB73FB7B3033FB73FB7B392B02D971
:1019E800FB7B0733FB73FB7B1846FFF79BFFFB79F9
:1019F80003F00F03FB73FB7B3033FB73FB7B392B4B
:101A080002D9FB7B0733FB73FB7B1846FFF78AFF82
:101A18002020FFF787FF00BF1037BD4680BD00BFFD
:101A280080B584B000AF0346FB71FB791B09FB73DB
:101A3800FB7B3033FB73FB7B392B02D9FB7B0733F2
:101A4800FB73FB7B1846FFF76DFFFB7903F00F0371
:101A5800FB73FB7B3033FB73FB7B392B02D9FB7B9E
:101A68000733FB73FB7B1846FFF75CFF00BF10379B
:101A7800BD4680BD80B584B000AF0346FB80FB88BF
:101A88001B0B9BB2DBB203F00F03FB73FB7B184607
:101A9800FFF76CFFFB881B0A9BB2DBB203F00F0356
:101AA800FB73FB7B1846FFF761FFFB881B099BB2A2
:101AB800DBB203F00F03FB73FB7B1846FFF756FFFF
:101AC800FB88DBB203F00F03FB73FB7B1846FFF7C1
:101AD8004DFF2020FFF726FF00BF1037BD4680BD11
:101AE80080B584B000AF78607B681B0FDBB203F071
:101AF8000F03FB73FB7B1846FFF738FF7B681B0E51
:101B0800DBB203F00F03FB73FB7B1846FFF72EFFD6
:101B18007B681B0DDBB203F00F03FB73FB7B1846DE
:101B2800FFF724FF7B681B0CDBB203F00F03FB738A
:101B3800FB7B1846FFF71AFF7B681B0BDBB203F031
:101B48000F03FB73FB7B1846FFF710FF7B681B0A2C
:101B5800DBB203F00F03FB73FB7B1846FFF706FFAE
:101B68007B681B09DBB203F00F03FB73FB7B184692
:101B7800FFF7FCFE7B68DBB203F00F03FB73FB7B14
:101B88001846FFF7F3FE2020FFF7CCFE00BF103702
:101B9800BD4680BD80B584B000AF78607B68002BFF
:101BA80005DA2D20FFF7BEFE7B685B427B607B6811
:101BB800092B40F2EE807B68632B40F2D2807B6871
:101BC800B3F57A7FC0F0B7807B6842F20F72934218
:101BD80040F29A807B68754A93427ED97B68744A42
:101BE800934263D97B68734A934249D97B68724AA6
:101BF80093422FD97B68714A934215D97B685B0A57
:101C08006F4AA2FB0323DB09FB60FB686D4A02FBFA
:101C180003F37A68D31A7B60FB68DBB23033DBB23C
:101C28001846FFF77FFE00E000BF7B68664AA2FB0C
:101C380003235B0EFB60FB68644A02FB03F37A68CC
:101C4800D31A7B60FB68DBB23033DBB21846FFF790
:101C580069FE00E000BF7B685D4AA2FB03239B0D81
:101C6800FB60FB685B4A02FB03F37A68D31A7B606C
:101C7800FB68DBB23033DBB21846FFF753FE00E0F7
:101C880000BF7B68544AA2FB03239B0CFB60FB68E4
:101C9800524A02FB03F37A68D31A7B60FB68DBB213
:101CA8003033DBB21846FFF73DFE00E000BF7B682B
:101CB8005B094B4AA2FB0323DB09FB60FB68494A2B
:101CC80002FB03F37A68D31A7B60FB68DBB230331C
:101CD800DBB21846FFF726FE00E000BF7B68424AE9
:101CE800A2FB03235B0BFB60FB6842F2107202FB52
:101CF80003F37A68D31A7B60FB68DBB23033DBB25C
:101D08001846FFF70FFE00E000BF7B68374AA2FBCA
:101D180003239B09FB60FB684FF47A7202FB03F311
:101D28007A68D31A7B60FB68DBB23033DBB21846C3
:101D3800FFF7F8FD00E000BF7B682D4AA2FB0323F4
:101D48005B09FB60FB68642202FB03F37A68D31A21
:101D58007B60FB68DBB23033DBB21846FFF7E2FD8D
:101D680000E000BF7B68234AA2FB0323DB08FB607B
:101D7800FA6813469B0013445B001A467B689B1A5B
:101D88007B60FB68DBB23033DBB21846FFF7CAFD75
:101D980000E000BF7B68DBB23033DBB21846FFF7E8
:101DA800C1FD00BF1037BD4680BD00BF9F86010042
:101DB8003F420F007F969800FFE0F505FFC99A3B68
:101DC800834B040000CA9A3B893BE65500E1F505C0
:101DD8006BCA5F6B8096980083DE1B4340420F00FE
:101DE800C55A7C0AA08601005917B7D1D34D621095
:101DF8001F85EB51CDCCCCCC80B582B000AF7860DC
:101E08007868FFF7C7FE2020FFF78CFD00BF083772
:101E1800BD4680BD80B582B000AF124B1B78002B49
:101E280011D1114B1B78002B0DD1104B1B78002BB7
:101E380009D003F081FD03461A46FA80002B02D030
:101E4800FB889BB20AE0FFF7F5FC03461A46FA80C6
:101E5800002B02D0FB889BB200E00023184608370D
:101E6800BD4680BDD01A0020824E0120773801205F
:101E780080B483B000AF3F4B1A683F4B1B689A424F
:101E880009D93D4B1B681A463A4B1B68D31A03F510
:101E9800AF537B6006E0384B1B681A46354B1B680E
:101EA800D31A7B607B6841F2D832934201D9002370
:101EB8005AE0324B1A68324B1B689A4209D9304BA8
:101EC8001B681A462D4B1B68D31A03F5AF537B606A
:101ED80006E02B4B1B681A46284B1B68D31A7B60FD
:101EE8007B6841F2D832934201D900233CE0254B6C
:101EF8001A68254B1B689A4209D9234B1B681A4656
:101F0800204B1B68D31A03F5AF537B6006E01E4BCA
:101F18001B681A461B4B1B68D31A7B607B6841F20F
:101F2800D832934201D900231EE0184B1A68184B87
:101F38001B689A4209D9164B1B681A46134B1B6833
:101F4800D31A03F5AF537B6006E0114B1B681A46A2
:101F58000E4B1B68D31A7B607B6841F2D8329342E0
:101F680001D9002300E0FF2318460C37BD465DF871
:101F7800047B70478C040020880400209C04002007
:101F880098040020AC040020A8040020BC04002011
:101F9800B804002080B400AF1F4B1B88002B0BD067
:101FA8001D4B1B881BB2002B06DB1B4B1B88013B00
:101FB8009AB2194B1A8002E0174B00221A80174B6D
:101FC8001B88002B05D0154B1B88013B9AB2134B7D
:101FD8001A80134B1B88002B05D0114B1B88013B23
:101FE8009AB20F4B1A800F4B1B88002B05D00D4B54
:101FF8001B88013B9AB20B4B1A800B4B1B88002B9A
:1020080005D0094B1B88013B9AB2074B1A8000BFC9
:10201800BD465DF8047B7047B0B40020CE1A00209E
:10202800D21A0020CC1A0020785C002080B400AFBF
:10203800204BDB6903F02003002B12D01E4B1B68DA
:102048005A1C1D490A601B4A928C92B2D2B21A706D
:10205800194B1A68194B1B689A4202D1164B184A39
:102068001A60144BDB6903F08003002B1ED0154B5C
:102078001A68154B1B689A4206D10E4A0D4B1B680D
:1020880023F08003136011E00A490E4B1B685A1CA9
:102098000C4802601B789BB20B850A4B1A680B4BE5
:1020A8001B689A4202D1074B094A1A60BD465DF87F
:1020B800047B704700380140800400202804002079
:1020C800107300208C040020880400202C040020B9
:1020D800EC04002080B400AF204BDB6903F0200340
:1020E800002B12D01E4B1B685A1C1D490A601B4A44
:1020F800928C92B2D2B21A70194B1A68194B1B689B
:102108009A4202D1164B184A1A60144BDB6903F045
:102118008003002B1ED0154B1A68154B1B689A427A
:1021280006D10E4A0D4B1B6823F08003136011E0A3
:102138000A490E4B1B685A1C0C4802601B789BB25C
:102148000B850A4B1A680B4B1B689A4202D1074B46
:10215800094A1A60BD465DF8047B70470048004094
:102168009004002030040020F08800209C04002007
:1021780098040020340400209846002080B400AF62
:10218800204BDB6903F02003002B12D01E4B1B6889
:102198005A1C1D490A601B4A928C92B2D2B21A701C
:1021A800194B1A68194B1B689A4202D1164B184AE8
:1021B8001A60144BDB6903F08003002B1ED0154B0B
:1021C8001A68154B1B689A4206D10E4A0D4B1B68BC
:1021D80023F08003136011E00A490E4B1B685A1C58
:1021E8000C4802601B789BB20B850A4B1A680B4B94
:1021F8001B689A4202D1074B094A1A60BD465DF82E
:10220800047B704700500040B004002040040020C8
:10221800B8300020BC040020B8040020440400208A
:10222800D09E002080B400AF204BDB6903F0200370
:10223800002B12D01E4B1B685A1C1D490A601B4AF2
:10224800928C92B2D2B21A70194B1A68194B1B6849
:102258009A4202D1164B184A1A60144BDB6903F0F4
:102268008003002B1ED0154B1A68154B1B689A4229
:1022780006D10E4A0D4B1B6823F08003136011E052
:102288000A490E4B1B685A1C0C4802601B789BB20B
:102298000B850A4B1A680B4B1B689A4202D1074BF5
:1022A800094A1A60BD465DF8047B7047004C00403F
:1022B800A004002038040020305D0020AC04002079
:1022C800A80400203C040020D41A002080B582B065
:1022D80000AF9F4B1B780133DAB29D4B1A709C4BB1
:1022E8001B78042B02D99A4B00221A70984B1B7842
:1022F800002B40F0D580974B1B78032B00F0878488
:102308000023FB71BBE0934B1B78012B07D103F033
:1023180013FB0346BB80BB88002B08D1B7E006F04F
:1023280077F80346BB80BB88002B00F0AD80BB88E4
:10233800FB7097F90330002B40DB874B1B88042B7D
:1023480009D100F037FD844B4FF4AF521A80834B0C
:102358004FF4AF521A80804B1B88002B00F09680F8
:102368007F4B1B78002B0ED07E4B1B685A1C7D4977
:102378000A607D4A11787D4A12780A43D2B21A70EF
:10238800774B00221A70774B1B685A1C75490A60F4
:10239800FA781A70704B1B88013B9AB26E4B1A8000
:1023A8006D4B1B88002B67D100F004FD6B4B1A881E
:1023B800694B1A806A4BFF221A7068E0684B00224A
:1023C8001A70FB78F72B10D1674B1B78F02B0CD1C8
:1023D800644B1B685A1C63490A60FA781A7000F04B
:1023E800E9FC5D4B00221A8051E0FB78F32B04D9FD
:1023F800FB78184600F0AEFC3EE05A4B5C4A1A6087
:10240800584B1B685A1C57490A60FA781A70524B85
:1024180000221A80FB7823F00F03DAB2524B1A70AD
:10242800FB7803F00F03DAB2504B1A70FB78F02BED
:1024380003D1494B4FF4AF521A80FB78F12B02D0ED
:10244800FB78F32B02D1444B01221A80464B1B78B0
:10245800C02B03D0444B1B78D02B02D13E4B01221A
:102468001A803D4B1B88002B02D13B4B02221A805D
:10247800394B1A88394B1A80FB790133FB71FB7988
:10248800022B7FF640AF02E000BF00E000BFFFF77D
:10249800EFFC0346002B00F0BC8300F095FFB8E387
:1024A8002B4B1B78012B40F0E6800023FB71D1E019
:1024B800FEF778FE0346BB80BB88002B00F0CF8078
:1024C800BB88FB7097F90330002B5FDB294B1B8817
:1024D800042B09D100F0CCFC264B4FF4AF521A80E4
:1024E800254B4FF4AF521A80224B1B88002B00F06B
:1024F800B880224B1B78002B0ED0214B1B685A1C2E
:102508001F490A601F4A11781F4A12780A43D2B23B
:102518001A701A4B00221A70194B1B685A1C18495A
:102528000A60FA781A70134B1B88013B9AB2114B58
:102538001A80104B1B88002B40F0898000F098FC13
:102548000D4B1A880B4B1A800C4BFF221A7089E02E
:10255800512201206C38012090E0002094E00020F6
:102568004038012098E00020A2CA00206C0C01200D
:10257800A4E0002062380120A0CA0020A3CA0020DD
:102588006438012093E000204E380120A44B00223B
:102598001A70FB78F72B13D1A24B1B78F02B0FD1B5
:1025A800A14B1B685A1CA0490A60FA781A7000F0FF
:1025B8005FFC9E4B00221A809D4B00221A8051E03E
:1025C800FB78F32B04D9FB78184600F0DBFB3EE0E0
:1025D800954B984A1A60944B1B685A1C92490A609A
:1025E800FA781A70914B00221A80FB7823F00F03B7
:1025F800DAB28C4B1A70FB7803F00F03DAB28E4B09
:102608001A70FB78F02B03D1884B4FF4AF521A8025
:10261800FB78F12B02D0FB78F32B02D1834B0122FC
:102628001A80804B1B78C02B03D07E4B1B78D02B95
:1026380002D17E4B01221A807C4B1B88002B02D1D1
:102648007A4B02221A80794B1A88794B1A80FB79C7
:102658000133FB71FB79022B7FF62AAF02E000BF42
:1026680000E000BFFFF704FC0346002B00F0D38214
:1026780000F0AAFECFE2714B1B78022B40F0C78016
:102688000023FB71B2E0FEF773FE0346BB80BB88F4
:10269800002B00F0B080BB88FB7097F90330002B4B
:1026A80040DB674B1B88042B09D100F03FFC644BCF
:1026B8004FF4AF521A80634B4FF4AF521A80604BFD
:1026C8001B88002B00F099805F4B1B78002B0ED0E5
:1026D8005E4B1B685A1C5D490A605D4A11785D4A69
:1026E80012780A43D2B21A70574B00221A70574B0D
:1026F8001B685A1C55490A60FA781A70504B1B8897
:10270800013B9AB24E4B1A804D4B1B88002B6AD165
:1027180000F00CFC4B4B1A88494B1A804A4BFF229D
:102728001A706BE0484B00221A70FB78F72B13D114
:10273800474B1B78F02B0FD1444B1B685A1C43495D
:102748000A60FA781A7000F0F1FB3D4B00221A80FB
:102758003C4B00221A8051E0FB78F32B04D9FB781C
:10276800184600F00FFB3EE0384B3B4A1A60374BE7
:102778001B685A1C35490A60FA781A70304B0022D7
:102788001A80FB7823F00F03DAB2314B1A70FB780A
:1027980003F00F03DAB22F4B1A70FB78F02B03D13A
:1027A800274B4FF4AF521A80FB78F12B02D0FB78FD
:1027B800F32B02D1224B01221A80254B1B78C02B08
:1027C80003D0234B1B78D02B02D11D4B01221A803A
:1027D8001B4B1B88002B02D1194B02221A80184B65
:1027E8001A88184B1A80FB790133FB71FB79022B8D
:1027F8007FF649AF02E000BF00E000BFFFF738FBFB
:102808000346002B00F0098200F0DEFD05E20B4BC9
:102818001B78032B40F0FA800023FB71E5E000BF32
:10282800A3CA002093E00020643801206238012008
:10283800A0CA002088F600204E380120512201202D
:102848006038012086F6002092E000205422012002
:10285800A0E000209EE00020B8B40020FEF7EAFFC8
:102868000346BB80BB88002B00F0C480BB88FB708C
:1028780097F90330002B40DB9D4B1B88042B09D1B3
:1028880000F0B2FB9A4B4FF4AF521A80994B4FF4B9
:10289800AF521A80964B1B88002B00F0AD80964BE8
:1028A8001B78002B0ED0954B1B685A1C93490A6065
:1028B800934A1178934A12780A43D2B21A708E4B0F
:1028C80000221A708D4B1B685A1C8C490A60FA78D2
:1028D8001A70874B1B88013B9AB2854B1A80844B30
:1028E8001B88002B7ED100F07FFB824B1A88804B1F
:1028F8001A80814BFF221A707FE07F4B00221A70EA
:10290800FB78F72B13D17E4B1B78F02B0FD17B4B29
:102918001B685A1C79490A60FA781A7000F064FB3F
:10292800734B00221A80734B00221A8065E0FB78F3
:10293800F32B18D9FB78184600F00CFA724B1B7869
:10294800002B4FD0714B1B78032B4BD0FB781846CC
:10295800FEF7FEFBFB781846FEF7E0FCFB7818460E
:10296800FEF7DCFD3EE0654B694A1A60634B1B6865
:102978005A1C62490A60FA781A705D4B00221A8064
:10298800FB7823F00F03DAB25D4B1A70FB7803F083
:102998000F03DAB25B4B1A70FB78F02B03D1544B60
:1029A8004FF4AF521A80FB78F12B02D0FB78F32B4F
:1029B80002D14F4B01221A80514B1B78C02B03D0F8
:1029C8004F4B1B78D02B02D1494B01221A80484B20
:1029D8001B88002B02D1464B02221A80444B1A88CE
:1029E800444B1A80FB790133FB71FB79022B7FF68C
:1029F80035AF02E000BF00E000BFFFF739FA034639
:102A0800002B00F00C8100F0DFFC08E1414B1B7843
:102A1800042B40F007810023FB71E7E0FEF7A8FDD7
:102A28000346BB80BB88002B00F0E580BB88FB70A9
:102A380097F90330002B41DB374B1B88042B09D156
:102A480000F0CAFB344B4FF4AF521A80334B4FF4AB
:102A5800AF521A80304B1B88002B00F0CE80304BD1
:102A68001B78002B0ED02F4B1B685A1C2D490A606F
:102A78002D4A11782D4A12780A43D2B21A70284B7F
:102A880000221A70274B1B685A1C26490A60FA78DC
:102A98001A70214B1B88013B9AB21F4B1A801E4BA0
:102AA8001B88002B40F09F8000F096FB1B4B1A8878
:102AB800194B1A801A4BFF221A709FE0184B0022FC
:102AC8001A70FB78F72B33D1174B1B78F02B2FD1CB
:102AD800144B1B685A1C13490A60FA781A7000F0E4
:102AE8007BFB0D4B00221A800C4B00221A8085E0DC
:102AF80050380120AACA002050220120C404002016
:102B08006B38012041380120A1E000206C380120F9
:102B1800ACCA0020512201206E380120443801201F
:102B28005C380120A4CA00209FE00020A8CA002029
:102B3800FB78F32B18D9FB78184600F00BF93B4BC0
:102B48001B78002B4FD03A4B1B78032B4BD0FB78CC
:102B58001846FEF7FDFAFB781846FEF7DFFBFB7810
:102B68001846FEF73DFE3EE0324B334A1A60314BC1
:102B78001B685A1C2F490A60FA781A702F4B0022DA
:102B88001A80FB7823F00F03DAB22D4B1A70FB780A
:102B980003F00F03DAB22B4B1A70FB78F02B03D13A
:102BA800264B4FF4AF521A80FB78F12B02D0FB78FA
:102BB800F32B02D1214B01221A80214B1B78C02B09
:102BC80003D01F4B1B78D02B02D11C4B01221A803B
:102BD8001A4B1B88002B02D1184B02221A80174B64
:102BE8001A88194B1A80FB790133FB71FB79022B88
:102BF8007FF614AF02E000BF00E000BFFFF738F92E
:102C08000346002B0DD000F0DFFB00BF09E000BF3A
:102C180008E000BF06E000BF04E000BF02E000BF1C
:102C280000E000BF0837BD4680BD00BF6A380120FC
:102C38006C380120A4CA0020700C01206E380120D5
:102C48009FE00020A8CA00204438012080B400AFCB
:102C5800264B274A1A60274B274A1A60274B284ACF
:102C68001A60284B284A1A60284B294A1A60294BAF
:102C7800294A1A60294B00221A80294B00221A80FF
:102C8800284B00221A80284B00221A80274B00224A
:102C98001A80274B00221A80264B9B6B1B0C9AB27A
:102CA800254B1A80234B9B6B9AB2244B1A80214BDD
:102CB800DB6B1B0C9AB2224B1A801E4BDB6B9AB251
:102CC800204B1A801B4B1B6C1B0C9AB21E4B1A8094
:102CD800184B1B6C9AB21D4B1A801D4B00221A70A0
:102CE80000BFBD465DF8047B704700BF6438012013
:102CF80088F6002054220120B8B40020C404002023
:102D0800ACCA0020A4CA0020700C012098E0002062
:102D1800A4E000209CCA0020602201206238012023
:102D280060380120503801206E38012090E00020E2
:102D380054380120D45C00205238012084F6002049
:102D4800B4B400204C3801205C22012068380120EE
:102D58005122012080B582B000AF0346FB71084BB9
:102D68001B78012B04D1FB79184605F029FA03E0FA
:102D7800FB79184602F060FE00BF0837BD4680BDEB
:102D88006C38012080B582B000AF0346FB71084B58
:102D98001B78022B04D1FB79184602F04DFE03E0A4
:102DA800FB79184605F00CFA00BF0837BD4680BD10
:102DB8006C38012080B582B000AF294B1B78012BFD
:102DC8002FD1284B284A1A600CE0264B1B6840F28A
:102DD800FC51184605F046FA224B1B6803F2FC53D7
:102DE800204A1360214B1B681A461E4B1B68D31AD6
:102DF80040F2FB529342E8DC1C4B1B681A46194B05
:102E08001B689A4225D0174B1A68184B1B6819463D
:102E1800144B1B68CB1A9BB21946104605F022FAD0
:102E280017E0124B1B681A460F4BD31AFB8000237E
:102E3800BB800BE0BB880C4AD35C184602F0FCFD53
:102E4800FB88013BFB80BB880133BB80FB88002BE0
:102E5800F0D1064B044A1A6000BF0837BD4680BD52
:102E68006C38012048380120A4E0002098E00020B8
:102E780080B582B000AF294B1B78022B18D1284BA4
:102E88001B681A46274BD31AFB800023BB800BE034
:102E9800BB88244AD35C184602F0CEFDFB88013B70
:102EA800FB80BB880133BB80FB88002BF0D12EE070
:102EB8001D4B1C4A1A600CE01B4B1B6840F2FC516E
:102EC800184605F0CFF9184B1B6803F2FC53164A55
:102ED8001360134B1B681A46134B1B68D31A40F236
:102EE800FB529342E8DC0E4B1B681A460E4B1B68DC
:102EF8009A420CD00C4B1A68094B1B6819460A4BAE
:102F08001B68CB1A9BB21946104605F0ABF9044B67
:102F1800044A1A6000BF0837BD4680BD6C380120DE
:102F28006438012088F6002098CA002080B582B055
:102F380000AF294B1B78022B18D1284B1B681A4667
:102F4800274BD31AFB800023BB800BE0BB88244AA5
:102F5800D35C184602F070FDFB88013BFB80BB8800
:102F68000133BB80FB88002BF0D12EE01D4B1C4A9F
:102F78001A600CE01B4B1B6840F2FC51184605F028
:102F880071F9184B1B6803F2FC53164A1360134B74
:102F98001B681A46134B1B68D31A1A4640F2FB5398
:102FA8009A42E7D80D4B1A680E4B1B689A420CD010
:102FB8000C4B1A68094B1B6819460A4B1B68CB1A3D
:102FC8009BB21946104605F04DF9044B044A1A60A5
:102FD80000BF0837BD4680BD6C380120542201204F
:102FE800B8B400208CE0002080B584B000AF724BEC
:102FF8001B681A46714BD31AFB81714B1B78012B46
:103008002FD1704B6D4A1A600CE06E4B1B6840F272
:10301800FC51184605F026F96A4B1B6803F2FC536D
:10302800684A1360644B1B681A46664B1B68D31AC0
:1030380040F2FB529342E8DC5F4B1B681A46614B37
:103048001B689A4221D05F4B1A685B4B1B68194674
:103058005C4B1B68CB1A9BB21946104605F002F967
:1030680013E0FB89BB8100237B810BE07B89534AFA
:10307800D35C184602F0E0FCBB89013BBB817B892D
:1030880001337B81BB89002BF0D14F4B1B78002B80
:1030980000F08A804A4B1B78032B00F085800023C0
:1030A8007B817DE07B89454AD35CBB71FB89013B11
:1030B800FB817B8901337B81BB79EF2B0ED9FF2301
:1030C800FB71BB791846FEF743F8BB791846FEF743
:1030D80025F9BB791846FEF721FA61E097F9063021
:1030E800002B2CDABB7903F00F03FB71FB79C3F1DA
:1030F8000F03012202FA03F33B81344B1A883B8900
:1031080013409BB2002B03D0BB791846FEF720F87A
:103118002F4B1A883B8913409BB2002B03D0BB79F5
:103128001846FEF7FBF82B4B1A883B8913409BB2D5
:10313800002B35D0BB791846FEF7F0F930E0FB7963
:10314800FF2B0CD1BB791846FEF702F8BB7918465D
:10315800FEF7E4F8BB791846FEF7E0F920E01B4BD0
:103168001A883B8913409BB2002B03D0BB791846C1
:10317800FDF7EEFF164B1A883B8913409BB2002BD4
:1031880003D0BB791846FEF7C9F8124B1A883B8959
:1031980013409BB2002B03D0BB791846FEF7BEF94B
:1031A800FB89002B7FF47EAF034B044A1A6000BFF3
:1031B8001037BD4680BD00BFC4040020ACCA002043
:1031C8006C380120C8040020A1E0002052380120FA
:1031D80084F600204C38012080B584B000AF724BD3
:1031E8001B681A46714BD31AFB81714B1B78012B54
:1031F8002FD1704B6D4A1A600CE06E4B1B6840F281
:10320800FC51184605F02EF86A4B1B6803F2FC5374
:10321800684A1360644B1B681A46664B1B68D31ACE
:1032280040F2FB529342E8DC5F4B1B681A46614B45
:103238001B689A4221D05F4B1A685B4B1B68194682
:103248005C4B1B68CB1A9BB21946104605F00AF86E
:1032580013E0FB89BB8100237B810BE07B89534A08
:10326800D35C184602F0E8FBBB89013BBB817B8934
:1032780001337B81BB89002BF0D14F4B1B78002B8E
:1032880000F08A804A4B1B78032B00F085800023CE
:103298007B817DE07B89454AD35CBB71FB89013B1F
:1032A800FB817B8901337B81BB79EF2B0ED9FF230F
:1032B800FB71BB791846FDF74BFFBB791846FEF743
:1032C8002DF8BB791846FEF78BFA61E097F90630BE
:1032D800002B2CDABB7903F00F03FB71FB79C3F1E8
:1032E8000F03012202FA03F33B81344B1A883B890E
:1032F80013409BB2002B03D0BB791846FDF728FF7B
:103308002F4B1A883B8913409BB2002B03D0BB7903
:103318001846FEF703F82B4B1A883B8913409BB2DB
:10332800002B35D0BB791846FEF75AFA30E0FB7906
:10333800FF2B0CD1BB791846FDF70AFFBB7918465D
:10334800FDF7ECFFBB791846FEF74AFA20E01B4B65
:103358001A883B8913409BB2002B03D0BB791846CF
:10336800FDF7F6FE164B1A883B8913409BB2002BDB
:1033780003D0BB791846FDF7D1FF124B1A883B8959
:1033880013409BB2002B03D0BB791846FEF728FAEE
:10339800FB89002B7FF47EAF034B044A1A6000BF01
:1033A8001037BD4680BD00BFA4CA0020700C0120A4
:1033B8006C380120583801206A3801205238012021
:1033C80084F60020B4B4002080B582B000AF684B0A
:1033D8001B78032B77D105F01BF80346FB80FB888D
:1033E800002B30D0FB887B717B79EF2B0BD9614B9D
:1033F800FF221A707B791846FDF7AAFE7B791846DA
:10340800FDF78CFF1FE097F90530002B0ADA7B796E
:1034180003F00F03DAB2574B1A707B79184600F0A5
:103428004FFA10E0534B1B78FF2B08D17B791846D5
:10343800FDF78EFE7B791846FDF770FF03E07B7978
:10344800184600F03DFA0023FB804B4B1B78002BFD
:1034580003D002F071FA0346FB80FB88002B00F0D2
:103468008380FB887B717B79EF2B0BD9414BFF2243
:103478001A707B791846FEF7B3F97B791846FEF780
:103488004DF871E097F90530002B0ADA7B7903F0E3
:103498000F03DAB2374B1A707B79184600F03EFA00
:1034A80062E0344B1B78FF2B08D17B791846FEF776
:1034B80097F97B791846FEF731F855E07B7918467D
:1034C80000F02CFA50E02A4B1B78012B04D104F0B1
:1034D8009FFF0346FB800DE0254B1B78022B09D18B
:1034E8000023FB80244B1B78002B03D002F024FA26
:1034F8000346FB80FB88002B37D0FB887B711F4B72
:103508001B78002B2BD11E4B1B78002B27D17B79E6
:10351800EF2B07D9174BFF221A707B79184600F05A
:103528003BF922E097F90530002B0ADA7B7903F0A2
:103538000F03DAB20F4B1A707B79184600F054F972
:1035480013E00C4B1B78FF2B04D17B79184600F055
:1035580023F90AE07B79184600F046F905E07B7903
:10356800184600F00FF800E000BF0837BD4680BDE0
:103578006C3801205822012077380120A1E0002072
:103588006A38012080B582B000AF0346FB7197F915
:103598000730002B40DB524B1B88042B09D100F06D
:1035A800ADF84F4B4FF4AF521A804E4B4FF4AF5219
:1035B8001A804B4B1B88002B00F08D804A4B1B78E0
:1035C800002B0ED0494B1B685A1C48490A60484AD0
:1035D8001178484A12780A43D2B21A70424B002234
:1035E8001A70424B1B685A1C40490A60FA791A70D3
:1035F8003B4B1B88013B9AB2394B1A80384B1B88CE
:10360800002B69D100F07AF8364B1A88344B1A80AF
:10361800354BFF221A705FE0334B00221A70FB799A
:10362800F72B10D1324B1B78F02B0CD12F4B1B688A
:103638005A1C2E490A60FA791A7000F05FF8284B74
:1036480000221A8048E0FB79F32B04D9FB7918464D
:1036580000F0A2F840E0254B274A1A60234B1B686C
:103668005A1C22490A60FA791A701D4B00221A80E6
:10367800FB7923F00F03DAB21D4B1A70FB7903F0C4
:103688000F03DAB21B4B1A70FB79F02B03D1144BE2
:103698004FF4AF521A80FB79F12B02D0FB79F32B50
:1036A80002D10F4B01221A80114B1B78C02B03D07B
:1036B8000F4B1B78D02B02D1094B01221A80084BE3
:1036C8001B88002B02D1064B02221A80044B1A8851
:1036D800044B1A8000E000BF0837BD4680BD00BF1C
:1036E800543801205E3801209CE000209CCA00204C
:1036F800A2E000205A2201206022012080B582B079
:1037080000AF224B1B681A46214BD31AFB800023BB
:10371800BB8030E0BB881E4AD35CFB70FB78EF2B84
:1037280007D91C4BFF221A70FB78184600F034F8B2
:103738001BE097F90330002B0ADAFB7803F00F033C
:10374800DAB2144B1A70FB78184600F04DF80CE00A
:10375800104B1B78FF2B04D1FB78184600F01CF89F
:1037680003E0FB78184600F03FF8FB88013BFB803C
:10377800BB880133BB80FB88002BCBD1034B044AA9
:103788001A6000BF0837BD4680BD00BF9CCA002034
:10379800602201205822012080B582B000AF034684
:1037A800FB71FB791846FDF7D3FCFB791846FDF74A
:1037B800B5FDFB791846FEF713F8FB791846FDF7B7
:1037C800ADFE084B1B78012B04D1FB79184602F09B
:1037D80033F903E0FB79184604F0F2FC00BF083720
:1037E800BD4680BD6C38012080B584B000AF03466B
:1037F800FB712B4B1B78C3F10F03012202FA03F371
:10380800FB81284B1A88FB8913409BB2002B03D0FD
:10381800FB791846FDF79CFC234B1A88FB8913405B
:103828009BB2002B03D0FB791846FDF777FD1F4BA1
:103838001A88FB8913409BB2002B03D0FB791846EA
:10384800FDF7CEFF1A4B1A88FB8913409BB2002B59
:1038580003D0FB791846FDF761FE164B1B78012B48
:103868000AD1154B1A88FB8913409BB2002B03D051
:10387800FB79184602F0E0F80E4B1B78022B0AD1B0
:103888000E4B1A88FB8913409BB2002B03D0FB799F
:10389800184604F095FC00BF1037BD4680BD00BF38
:1038A800582201205238012084F60020B4B40020A8
:1038B8004C3801206C380120683801205C22012036
:1038C80080B584B000AF0346FB71114B1B78C3F180
:1038D8000F03012202FA03F3FB810E4B1A88FB89BE
:1038E80013409BB2002B03D0FB791846FDF730FC40
:1038F800094B1A88FB8913409BB2002B03D0FB7934
:103908001846FDF70BFD00BF1037BD4680BD00BF50
:10391800582201205238012084F6002080B584B056
:1039280000AF0346FB71114B1B78C3F10F03012253
:1039380002FA03F3FB810E4B1A88FB8913409BB2F2
:10394800002B03D0FB791846FDF74AFF094B1A886C
:10395800FB8913409BB2002B03D0FB791846FDF777
:10396800DDFD00BF1037BD4680BD00BF58220120D5
:10397800B4B400204C38012080B582B000AFA44B0D
:103988001B780133DAB2A24B1A70A14B1B78022BB9
:1039980002D99F4B00221A709D4B1B78002B40F0D8
:1039A800DE800023FB71B2E0FDF7FCFB0346BB8021
:1039B800BB88002B00F0B080BB88FB7097F9033000
:1039C800002B40DB934B1B88042B09D1FFF750FADF
:1039D800904B4FF4AF521A808F4B4FF4AF521A806E
:1039E8008C4B1B88002B00F099808C4B1B78002B8C
:1039F8000ED08B4B1B685A1C89490A60894A11787A
:103A0800894A12780A43D2B21A70844B00221A707B
:103A1800834B1B685A1C82490A60FA781A707D4BDE
:103A28001B88013B9AB27B4B1A807A4B1B88002B70
:103A38006AD100F0BDFA784B1A88764B1A80774B1A
:103A4800FF221A706BE0754B00221A70FB78F72B77
:103A580013D1744B1B78F02B0FD1714B1B685A1C78
:103A68006F490A60FA781A7000F0A2FA694B0022CE
:103A78001A80694B00221A8051E0FB78F32B04D995
:103A8800FB781846FDF74AFD3EE0654B674A1A6029
:103A9800634B1B685A1C62490A60FA781A705D4BBE
:103AA80000221A80FB7823F00F03DAB25D4B1A70FC
:103AB800FB7803F00F03DAB25B4B1A70FB78F02B3C
:103AC80003D1544B4FF4AF521A80FB78F12B02D03C
:103AD800FB78F32B02D14F4B01221A80514B1B78F4
:103AE800C02B03D04F4B1B78D02B02D1494B01225E
:103AF8001A80484B1B88002B02D1464B02221A80A1
:103B0800444B1A88444B1A80FB790133FB71FB79CB
:103B1800022B7FF649AF02E000BF00E000BFFDF7CF
:103B280027FD0346BB80BB88002B00F02B82BB8897
:103B3800FB70FB781846FDF70BFBFB781846FDF782
:103B4800EDFB3B4B1B78032B04D1FB78184601F0A7
:103B580073FF17E2FB78184604F032FB12E22C4B95
:103B68001B78012B40F0FE800023FB71D2E0FDF7AB
:103B7800FFFB0346BB80BB88002B00F0D080BB88CE
:103B8800FB7097F90330002B60DB2A4B1B88042B52
:103B980009D1FFF7CBF9274B4FF4AF521A80264BC8
:103BA8004FF4AF521A80234B1B88002B00F0B980CA
:103BB800224B1B78002B0ED0214B1B685A1C204926
:103BC8000A60204A1178204A12780A43D2B21A7041
:103BD8001A4B00221A701A4B1B685A1C18490A60A3
:103BE800FA781A70134B1B88013B9AB2114B1A8052
:103BF800104B1B88002B40F08A8000F0FFF90E4B19
:103C08001A880C4B1A800D4BFF221A708AE000BFED
:103C18005122012062380120A0CA0020A3CA002036
:103C28006438012093E000204E38012088F60020F7
:103C3800D01A00206038012086F6002092E000208B
:103C480054220120A0E000209EE00020884B0022A2
:103C58001A70FB78F72B13D1864B1B78F02B0FD1FA
:103C6800854B1B685A1C84490A60FA781A7000F060
:103C7800C5F9824B00221A80814B00221A8051E03C
:103C8800FB78F32B04D9FB781846FDF747FC3EE098
:103C9800794B7C4A1A60784B1B685A1C76490A6033
:103CA800FA781A70754B00221A80FB7823F00F03FC
:103CB800DAB2704B1A70FB7803F00F03DAB2724B6A
:103CC8001A70FB78F02B03D16C4B4FF4AF521A806B
:103CD800FB78F12B02D0FB78F32B02D1674B012242
:103CE8001A80644B1B78C02B03D0624B1B78D02BF7
:103CF80002D1624B01221A80604B1B88002B02D133
:103D08005E4B02221A805D4B1A885D4B1A80FB7944
:103D18000133FB71FB79022B7FF629AF02E000BF6C
:103D280000E000BFFDF724FC0346BB80BB88002BE6
:103D380000F02A81BB88FB70FB781846FDF708FA6B
:103D4800FB781846FDF7EAFA504B1B78032B04D191
:103D5800FB78184601F070FE16E1FB78184604F06F
:103D68002FFA11E14A4B1B78022B40F010810023F7
:103D7800FB71DFE0454B1B78032B07D101F0DCFD1D
:103D88000346BB80BB88002B08D1DBE004F040FB76
:103D98000346BB80BB88002B00F0D180BB88FB703A
:103DA80097F90330002B41DB3A4B1B88042B09D1D0
:103DB800FFF700F8374B4FF4AF521A80364B4FF4E9
:103DC800AF521A80334B1B88002B00F0BA80334B5C
:103DD8001B78002B0ED0324B1B685A1C30490A60E6
:103DE800304A1178304A12780A43D2B21A702B4BF3
:103DF80000221A702D4B1B685A1C2C490A60FA784D
:103E08001A70244B1B88013B9AB2224B1A80214B13
:103E18001B88002B40F08B8000F016F91E4B1A8887
:103E28001C4B1A801D4BFF221A708BE01B4B002283
:103E38001A70FB78F72B13D11A4B1B78F02B0FD184
:103E48001A4B1B685A1C19490A60FA781A7000F054
:103E5800FBF8104B00221A800F4B00221A8071E0E9
:103E6800FB78F32B24D9FB781846FDF757FB5EE067
:103E780092E00020A0E000205422012060380120B8
:103E880086F60020B8B400209EE00020D01A00205A
:103E98005122012090E0002094E0002040380120C9
:103EA80064380120A2CA00206C0C012098E0002090
:103EB800384B394A1A60374B1B685A1C35490A6017
:103EC800FA781A70354B00221A80FB7823F00F031A
:103ED800DAB2334B1A70FB7803F00F03DAB2314BC6
:103EE8001A70FB78F02B03D12C4B4FF4AF521A8089
:103EF800FB78F12B02D0FB78F32B02D1274B012260
:103F08001A80274B1B78C02B03D0254B1B78D02B4E
:103F180002D1224B01221A80204B1B88002B02D190
:103F28001E4B02221A801D4B1A881F4B1A80FB79E0
:103F38000133FB71FB79022B7FF61CAF02E000BF57
:103F480000E000BFFDF714FB0346BB80BB88002BD5
:103F58001CD0BB88FB70FB781846FDF7F9F8FB7896
:103F68001846FDF7DBF9114B1B78032B04D1FB78BE
:103F7800184601F061FD09E0FB78184604F020F9C5
:103F880000BF03E000BF02E000BF00E000BF083749
:103F9800BD4680BD98E00020A4E0002090E000200D
:103FA800A2CA00206C0C012094E00020D01A002046
:103FB80080B582B000AF0F4B1B681A460E4BD31A60
:103FC800FB800023BB800BE0BB880B4AD35C184600
:103FD800FDF7A4FAFB88013BFB80BB880133BB805B
:103FE800FB88002BF0D1034B034A1A6000BF083747
:103FF800BD4680BD6438012088F6002080B582B0B7
:1040080000AF0F4B1B681A460E4BD31AFB800023D8
:10401800BB800BE0BB880B4AD35C1846FDF77EFAE1
:10402800FB88013BFB80BB880133BB80FB88002BEE
:10403800F0D1034B034A1A6000BF0837BD4680BD64
:1040480054220120B8B4002080B582B000AF0F4BD5
:104058001B681A460E4BD31AFB800023BB800BE06B
:10406800BB880B4AD35C1846FDF758FAFB88013B1E
:10407800FB80BB880133BB80FB88002BF0D1034B4E
:10408800034A1A6000BF0837BD4680BD98E000208B
:10409800A4E00020DFF834D0002103E00C4B5B588B
:1040A800435004310B480C4B42189A42F6D30B4A42
:1040B80002E0002342F8043B094B9A42F9D300F08E
:1040C80013F8FCF78BF8FCF78DF9FEE70080012068
:1040D800D493000800000020640400206404002039
:1040E8007C760120FEE7000080B400AF174A174B2A
:1040F800D3F8883043F47003C2F88830144A144B5C
:104108001B6843F001031360114B00229A60104AA8
:104118000F4B1B6823F0A85323F4102313600C4B98
:104128004FF48052DA600A4A094B1B6823F4802353
:104138001360074B00229A61044B4FF000629A60AB
:1041480000BFBD465DF8047B704700BF00ED00E08E
:104158000010024080B483B000AF0346FB710949E8
:1041680097F907305B09FA7902F01F02012000FA7B
:1041780002F241F8232000BF0C37BD465DF8047BEE
:10418800704700BF00E100E080B483B000AF034691
:10419800FB71094997F907305B09FA7902F01F02A8
:1041A800012000FA02F2203341F8232000BF0C3727
:1041B800BD465DF8047B704700E100E080B500AFC4
:1041C800224B00221A70224A214B5B6843F00203FB
:1041D80053603220FCF73CFB4FF090424FF0904385
:1041E8005B6A23F47F2323F0F00353624FF090427D
:1041F8004FF090431B6823F0A27313604FF0904276
:104208004FF090431B6823F0227313604320FFF79D
:10421800BBFF104A0F4BDB6A43F48053D3620E4A4C
:104228000D4B1B6843F0130313604FF0A0424FF08F
:10423800A0439B6B23F480339363064A054BDB6CE6
:1042480023F48053D36400BF80BD00BF77380120BA
:104258000008005000100240000E005080B500AF6A
:104268007A4A7A4BDB6A43F48053D362774A774BB6
:10427800DB6A23F48053D362744A744BDB6C23F4F7
:104288008053D364724A724B5B6843F48063536013
:104298004FF090424FF090431B6823F44023136083
:1042A8004FF090424FF09043DB6823F44023D360F3
:1042B8004FF090424FF090435B6A23F47F235362A0
:1042C8004FF090424FF090435B6A43F42A235362C5
:1042D8004FF090424FF090431B6823F0A073136097
:1042E8004FF090424FF090431B6843F020731360E7
:1042F8004FF090424FF090439B6823F070739360A7
:104308004FF090424FF090439B6843F0A073936046
:104318004FF090424FF09043DB6823F07073D36006
:104328004A4A4A4BDB6C43F48053D3644FF0A042B3
:104338004FF0A0439B6823F001039360454B032291
:104348001A6000BF4FF0A0431B69002BFADA4FF048
:10435800A0424FF0A0431B6943F001031361012001
:10436800FCF776FA00BF4FF0A0431A693A4B1340A6
:10437800B3F1004FF7D10120FCF76AFA354A354B03
:104388005B6823F0020353600220FCF761FA4FF0E8
:1043980090424FF090431B6823F4402313604FF082
:1043A80090424FF09043DB6823F44023D3604FF0F2
:1043B800A0434FF404129A633220FCF749FA4FF0F5
:1043C800A0424FF0A043DB6843F0804343F4C2535C
:1043D800D3603220FCF73CFA4FF0A0434FF0FF3295
:1043E8005A614FF0A0431D4A9A611D4B00221A6082
:1043F800184B00221A61174B00225A61154B0022F4
:10440800DA6100F02FF800BF4FF0A0435B6923F496
:104418000053002BF8D000BF4FF0A0435B6923F492
:104428008053002BF8D04FF0A0424FF0A0435B69B7
:1044380043F440535361074A064B5B6843F4807367
:1044480053604320FFF786FE00BF80BD0010024086
:10445800007000400008005001000080083C008007
:10446800000E005080B400AF7C4B00221A707C4BC9
:1044780003221A604FF0A04380225A62794B7A4A8D
:104488001A607A4B7A4A1A607A4B00221A607A4B81
:104498001B78002B02D1794B794A1A604FF0A04261
:1044A8004FF0A0431B6943F03003136100BF4FF086
:1044B800A0431B6903F03003002BF8D1714B002295
:1044C8001A60714A704B1B6843F05B0313606F4BB3
:1044D80000221A606E4B4FF000421A606D4A6D4B15
:1044E8001B6843F05B0313606B4B6C4A1A606C4BA0
:1044F8006C4A1A606C4A6C4B1B6843F05B03136090
:104508006A4B00221A606A4B4FF480021A60694AAB
:10451800684B1B6843F05B031360674B00221A600B
:10452800664B4FF400021A60654A654B1B6843F0FE
:104538005B031360634B00221A60634B634A1A6083
:10454800634A634B1B6843F05B031360614B624A29
:104558001A60494B1B78002B19D1604B604A1A60CE
:10456800604A604B1B6843F05B0313605E4B00229C
:104578001A605E4B4FF440021A605D4A5C4B1B6840
:1045880043F05B0313605B4B00221A6017E0534B48
:1045980000221A60534A534B1B6843F05B031360B5
:1045A800514B00221A60514B00221A60504A504B5E
:1045B8001B6843F05B0313604E4B00221A60284AC5
:1045C800274B5B6943F009035361254A244B1B6958
:1045D80043F0190313614FF0A04300229A614FF092
:1045E800A0434FF0FF325A614FF0A0414FF0A04373
:1045F8009A69414B13438B614FF0A0424FF0A0439F
:104608009B6843F081039360154B3C4ADA611A4B6F
:104618001B78002B05D1124A114BDB6943F00803C4
:10462800D3610F4B00225A63354B00221A70354B69
:1046380000221A80344B354A1A60354B334A1A60C7
:10464800344B354A1A60354B334A1A60344B0022D2
:104658001A7000BFBD465DF8047B704777380120AB
:10466800000800502800005080004000040100505D
:104678000001400008010050824E01200C0100504A
:10468800800120000009005008090050100900505E
:10469800000B0050080B0050100B00504000086041
:1046A80020090050400048002809005030090050F7
:1046B800200B0050280B0050300B005040090050D0
:1046C8004809005050090050400B00504000880035
:1046D800480B0050500B0050400008006009005083
:1046E8001000CC006809005070090050600B0050A1
:1046F800680B0050700B005018380C0003000500C0
:104708007238012074380120CC0400209C38012024
:10471800D0040020D40400208C4E0120D8040020AE
:10472800814E012080B582B000AF4FF0A0435A6996
:104738004FF0A0439B6913407B607B68002B46D0F9
:104748007B6803F48023002B01D000F0CFFA7B684C
:1047580003F40023002B01D000F08EFC7B6803F0EB
:104768001003002B01D000F037F87B6803F0080332
:10477800002B03D04FF0A04308225A617B6803F452
:104788008053002B06D0FFF76DFE4FF0A0434FF487
:1047980080525A617B6803F40053002B04D04FF019
:1047A800A0434FF400525A617B68002B04DA4FF0A3
:1047B800A0434FF000425A617B6803F40063002B6A
:1047C80006D04FF0A0434FF400625A6100E000BFEA
:1047D8000837BD4680BD00BF80B586B000AF4FF03A
:1047E800A0424FF0A0439B6923F0100393619B4BB9
:1047F8007B614FF0A0431B6AFB60FA68984B13403B
:10480800BB60FB6803F00F03002B3ED1BB68BB689D
:10481800944A93420ED17B691B68BB607B691B6815
:104828007B60914B20221A70904B00221A80904B8B
:10483800FF221A70FB6803F4F013B3F5402F24D15C
:104848007B691B68BB607B691B687B60BB68DAB2ED
:10485800884B1A70BB681B0ADAB2874B1A70BB68A0
:104868001B0C9AB2854B1A80844B1B889BB21B0A7F
:104878009BB2DAB2824B1A707B689AB2814B1A806B
:104888007B681B0C9AB2804B1A80FA687F4B1340E6
:104898007F4A934240F0D580FB6803F47F631B098D
:1048A800DAB27C4B1A708CE07B691B68BB607A4B70
:1048B8001B78012B04D1BB68184600F0FBF880E098
:1048C800BB68FB74754B1B685A1C74490A60FA7CF8
:1048D8001A70724B1A68724B1B689A4202D16F4B5E
:1048E800704A1A606B4B1B78DBB2013BDAB2694B3A
:1048F8001A70684B1B78DBB2002B75D0BB6803F4C9
:104908007F431B0AFB74654B1B685A1C63490A608A
:10491800FA7C1A70614B1A68614B1B689A4202D183
:104928005E4B604A1A605B4B1B78DBB2013BDAB224
:10493800584B1A70574B1B78DBB2002B56D0BB680C
:1049480003F47F031B0CFB74544B1B685A1C53491C
:104958000A60FA7C1A70514B1A68514B1B689A42CC
:1049680002D14E4B4F4A1A604A4B1B78DBB2013BCF
:10497800DAB2484B1A70474B1B78DBB2002B37D0A2
:10498800BB6803F07F431B0EFB74444B1B685A1C27
:1049980042490A60FA7C1A70404B1A68404B1B68FF
:1049A8009A4202D13D4B3F4A1A603A4B1B78DBB220
:1049B800013BDAB2374B1A70364B1B78DBB2002B4F
:1049C80018D0344B1B78DBB21946334B1B781A4688
:1049D80013465B00134499420DDD2E4B1B78DBB266
:1049E800402B7FF661AF06E000BF04E000BF02E0A5
:1049F80000BF00E000BF2C4B1A68284B1B689A4286
:104A080009D9264B1B6803F5AF531A46264B1B687A
:104A1800D31A3B6006E0214B1B681A46224B1B68E1
:104A2800D31A3B60214B00221A703B6841F2DC42EA
:104A3800934206D91D4BFF221A701D4B4FF40022DA
:104A48009A614FF0A0424FF0A0439B6943F01003D6
:104A5800936100BF1837BD4680BD00BF00100050ED
:104A6800FF7F1E0070000400723801207438012096
:104A780077380120853801207E4E012080380120BA
:104A88008A4E0120884E0120783801200F001E0030
:104A980002000400854E0120824E0120D40400202B
:104AA8005C0400208C4E0120D8040020844E012094
:104AB8000008004880B485B000AF78607B68FB735D
:104AC800834B1B78DBB2013BDAB2814B1A70804B07
:104AD8001B78DBB2002B00F0E1807B681B0ABB73FC
:104AE8007B4B1B78DBB2013BDAB2794B1A70784BFF
:104AF8001B78DBB2002B00F0D3807B681B0C7B7328
:104B0800734B1B78DBB2013BDAB2714B1A70704BF6
:104B18001B78DBB2002B00F0C5807B681B0E3B7353
:104B28006B4B1B78DBB2013BDAB2694B1A70FB7B2B
:104B38000F2B00F2B980FB7B012B40F2B780FB7B87
:104B4800052B02D0FB7B0F2B29D1BB7BF82B04D183
:104B5800604B1B78002B40F0AB80BB7BFE2B04D155
:104B68005D4B1B78002B40F0A580BB7BF62B04D156
:104B78005A4B1B78002B40F09F80594B1B685A1CDE
:104B880057490A60BA7B1A70554B1A68554B1B680F
:104B98009A4240F09380524B534A1A608EE0FB7B56
:104BA8000C2B02D0FB7B0D2B20D14D4B1B685A1CC4
:104BB8004B490A60BA7B1A70494B1A68494B1B6803
:104BC8009A4202D1464B484A1A60454B1B685A1C08
:104BD80043490A607A7B1A70414B1A68414B1B683B
:104BE8009A426DD13E4B404A1A6069E0FB7B022B2A
:104BF80002D0FB7B062B20D1394B1B685A1C384945
:104C08000A60BA7B1A70364B1A68364B1B689A4290
:104C180002D1334B344A1A60314B1B685A1C304955
:104C28000A607A7B1A702E4B1A682E4B1B689A42C0
:104C380048D12B4B2C4A1A6044E0294B1B685A1C5C
:104C480027490A60BA7B1A70254B1A68254B1B68DE
:104C58009A4202D1224B244A1A60214B1B685A1CE3
:104C68001F490A607A7B1A701D4B1A681D4B1B6816
:104C78009A4202D11A4B1C4A1A60194B1B685A1CDB
:104C880017490A603A7B1A70154B1A68154B1B684E
:104C98009A4218D1124B144A1A6014E000BF12E06D
:104CA80000BF10E000BF0EE000BF0CE000BF0AE04C
:104CB80000BF08E000BF06E000BF04E000BF02E05C
:104CC80000BF00E000BF1437BD465DF8047B7047A5
:104CD800854E012042380120592201209DE0002004
:104CE800D40400205C0400208C4E012080B582B0E2
:104CF80000AF784B9B69DAB2764BDB69DBB21340C5
:104D0800DBB2FB71FB79DBB203F00103002B00F08F
:104D18008780704B1A696F4B5B6B03F00103DB01F3
:104D280013433B606C4B1A683B6813403B603B681D
:104D380003F08003002B11D0664A664B5B6B23F0AF
:104D480001035363654B1B78DBB2062B04D0634B1E
:104D58001B78DBB2A12B01D100F01AFC3B6803F0F1
:104D68000103002B4CD05C4B01221A605C4B1B8862
:104D78009BB2002B31D1594B1B78DBB2052B06D0E7
:104D8800564B1B78DBB2092B01D0544B1B78534B85
:104D98001B78DBB2202B10D1524B1B78002B0CD187
:104DA800514B524A1A60524B524A1A60524B1B7866
:104DB800002B02D1514B524A1A60464A454B5B6B55
:104DC80023F0010353634F4B4F4A1A604F4A4F4B2E
:104DD8001B6843F00443136012E04D4B404A1288AD
:104DE80092B242F400221A604A4A4A4B1B6843F0C6
:104DF80004431360374A374B5B6B43F0010353633B
:104E08003B6803F01003002B02D0334B10221A60CA
:104E18003B6803F00803002B02D02F4B08221A60CE
:104E2800FB79DBB203F00203002B00F0B180294BC1
:104E38001A69284B5B6B03F002039B0113433B6029
:104E4800354B1A683B6813403B603B6803F08003AE
:104E5800002B07D01F4A1F4B5B6B23F002035363E1
:104E680000F00AFC3B6803F00103002B05D13B6806
:104E780003F01003002B00F083803B6803F001036C
:104E8800002B02D0244B01221A60244B1A68244BB1
:104E98001B689A420CD1144A134B1B6843F0044315
:104EA80013600C4A0B4B5B6B23F0020353635FE008
:104EB8001A4B1A681A4B1B689A4235D9184B1B684B
:104EC80003F5AF531A46154B1B68D31A9AB2154B04
:104ED8001A8032E00008005008090050723801209A
:104EE8007438012077380120200900504080488418
:104EF800400B005040808884824E01206009005099
:104F08001080CC84100B005040000860000B00504B
:104F1800100900500009005028090050D004002052
:104F2800CC04002070380120494B1B681A46494BB5
:104F38001B68D31A9AB2484B1A80474B1B889BB2FE
:104F4800402B02D9444B40221A80444B424A1288D3
:104F580092B242F400221A60414A414B1B6843F066
:104F6800044313603F4A3F4B5B6B43F002035363B8
:104F78003B6803F01003002B02D03B4B10221A6051
:104F88003B6803F00803002B02D0374B08221A6055
:104F9800FB79DBB203F00803002B54D0314B1A69BC
:104FA800304B5B6B03F008031B0113433B602F4B33
:104FB8001A683B6813403B603B6803F08003002B92
:104FC80009D02B4B4FF400221A602A4A294B1B6840
:104FD80043F0044313603B6803F00103002B12D035
:104FE800234B4FF400221A60224A224B1B6843F0DD
:104FF800044313601D4B01221A601A4A194B5B6B5C
:1050080023F0080353633B6803F01003002B12D00E
:10501800174B4FF400221A60164A164B1B6843F0D0
:10502800044313600F4A0F4B5B6B23F00803536371
:105038000E4B10221A603B6803F00803002B02D0C5
:105048000A4B08221A6000BF0837BD4680BD00BF62
:10505800CC040020D0040020703801203009005012
:105068002009005000080050280900506809005025
:10507800700900506009005080B582B000AF6D4BD8
:105088009A696C4BDB6913401B0CDBB2FB71FB7933
:10509800DBB203F00103002B00F09B80664B1B681A
:1050A800DAB2644B5B69DBB21340DBB2BB71BB792C
:1050B800DBB203F00103002B1AD05F4B01221A6008
:1050C8005E4B5F4A1A605F4A5E4B1B6843F00443BD
:1050D80013605D4B1B78DBB2202B09D15B4B4FF47F
:1050E80000221A605A4A5A4B1B6843F00443136063
:1050F800BB79DBB203F00803002B00F0978000F0C7
:10510800B7F8514B1B78DBB2052B1BD1514B1B78E1
:10511800DBB21901474A474B1B680B4313604B4BE3
:105128004FF400221A604A4A494B1B6843F0044373
:105138001360414B08221A603E4A3E4B5B6B43F0BA
:1051480001035363404B1B78DBB2092B04D03E4B61
:105158001B78DBB2222B12D13C4B4FF400221A6091
:105168003B4A3B4B1B6843F004431360324B082215
:105178001A60304A2F4B5B6B43F001035363324B89
:105188001B78DBB2062B04D02F4B1B78DBB2A12B8C
:105198004CD1314B1B889BB2402B03D92B4B2F4A48
:1051A8001A6006E0294B2C4A128892B242F4002277
:1051B8001A60274A264B1B6843F0044313601E4BB2
:1051C80008221A601B4A1B4B5B6B43F001035363B5
:1051D8002CE0FB79DBB203F00403002B27D0204B33
:1051E8001B68DAB2134B5B69DBB21340DBB2BB71ED
:1051F800BB79DBB203F00103002B18D0184B012256
:105208001A60184B154A1A60174B1B78002B06D1E9
:10521800164A164B1B6843F00443136007E0134A11
:10522800124B1B6843F00043136000E000BF0837CF
:10523800BD4680BD00080050080B0050100B005000
:1052480040000860000B005072380120100900501F
:10525800000900509A3801207438012040000800E5
:10526800480B0050500B0050844E0120400B00505A
:1052780080B582B000AF924B00221A70914B1B7818
:10528800DBB2212B29D1904B1B78DBB2202B12D11A
:105298008E4A8E4B1B6843F0080313608C4B8D4A73
:1052A8001A608D4A8C4B1B6843F004431360844B8F
:1052B80020221A7054E1844B1B78DBB2222B09D1CF
:1052C8007F4B22221A70854B00221A80844BFF22C2
:1052D8001A7045E100F0C0F942E17A4B1B78DBB265
:1052E800A12B1BD1784B1B78DBB2212B16D1744B29
:1052F800A1221A70794B07221A807A4B1B889AB21E
:10530800764B1B889BB29A4204D2764B1B889AB282
:10531800724B1A80744B754A1A6021E1694B1B78ED
:10532800DBB203F06103002B07D0664B1B78DBB2BE
:1053380003F06103012B40F01181634B1B78DBB252
:10534800092B00F2028101A252F823F059550008F6
:105358005355000853550008535500085355000885
:105368007D5300089D530008535500085355000805
:10537800255500085E4B1B889BB2DBB203F07F0308
:10538800DAB25C4B1A704E4B05221A70534B00224E
:105398001A80E2E04A4B06221A70574B1B78DBB2A0
:1053A800012B4DD14D4B12221A80544B1B78012BE7
:1053B80003D14D4B524A1A6002E04B4B514A1A60D6
:1053C800514B3B600023FB800CE03B685A1C3A6061
:1053D800454A1268511C4448016012781A70FB88CB
:1053E8000133FB80FB88112BEFD9484B1A68474BD8
:1053F8005B681343002B1FD0444B1B68DAB2424B47
:105408001A72424B1B681B0ADAB23F4B5A723F4B67
:105418005B68DAB23C4B9A723C4B5B681B0ADAB2A7
:10542800394BDA72354B1B78012B05D1364B9B7AF9
:105438000133DAB2344B9A722B4B334A1A6089E043
:105448002D4B1B78DBB2022B1ED12C4B1B78012B6A
:1054580006D1224B65221A80234B2D4A1A6005E09B
:105468001E4B43221A80204B2A4A1A601D4B1B8868
:105478009AB21A4B1B889BB29A426BD2194B1B8863
:105488009AB2164B1A8065E01B4B1B78DBB2032BD4
:1054980013D1124B18221A80124B1B889AB20F4B49
:1054A8001B889BB29A4204D20E4B1B889AB20B4BB4
:1054B8001A800D4B184A1A604CE000F0CDF849E00C
:1054C80072380120853801207E4E0120080B0050DB
:1054D800100B005040000860000B00507438012089
:1054E80077380120783801207C380120F88D0008B1
:1054F800803801209A3801208A4E0120824E0120EE
:10550800008E0008888D000888380120D45C0020AF
:10551800148E00089C8D0008E08D0008124B0922AB
:105528001A70124B00221A80114BFF221A70114B6D
:10553800114A1A60114B124A1A60124B1B78002B41
:105548000AD1114B114A1A6006E000F085F804E010
:1055580000BF05E000BF03E000BF01E000F07CF8F9
:105568000837BD4680BD00BF72380120743801205D
:10557800773801202009005040804884400B0050B3
:1055880040808884824E0120600900501080CC84BD
:1055980080B485B000AF2D4B1B889BB2402B11D92E
:1055A8002B4B1B68FB602A4B1B684033284A13604F
:1055B8004023FB70254B1B889BB2403B9AB2234B80
:1055C8001A800AE0224B1B68FB60204B1B889BB2A9
:1055D800DBB2FB701D4B00221A80FB78DBB2033371
:1055E800002B00DA03339B10DBB2BB70194BBB6096
:1055F80000237B701DE0FB6803331B781B061A46EB
:10560800FB6802331B781B041343FA6801321278D3
:1056180012021343FA68127813437B607A68BB68F6
:105628001A60FB680433FB607B78DBB20133DBB2C2
:105638007B707B78DAB2BB78DBB29A42DBD300BFEF
:105648001437BD465DF8047B704700BF74380120ED
:105658007C3801200010005080B400AF054A054B8B
:105668001B6843F40013136000BFBD465DF8047B5C
:10567800704700BF000B005080B487B000AF514B9B
:105688007B61514B1B683B618AE0504B1B681B7860
:10569800DBB2FB604D4B1B6801334C4A13604B4B2C
:1056A8001A684B4B1B689A4202D1484B494A1A6008
:1056B800494B1B889BB2013B9AB2474B1A80002387
:1056C800BB6000237B6000233B60434B1B889BB27D
:1056D800002B19D03D4B1B681B78DBB2BB603B4BE2
:1056E8001B680133394A1360384B1A68384B1B68FA
:1056F8009A4202D1354B374A1A60374B1B889BB206
:10570800013B9AB2344B1A80334B1B889BB2002B57
:1057180019D02E4B1B681B78DBB27B602B4B1B68A8
:1057280001332A4A1360294B1A68294B1B689A428D
:1057380002D1264B274A1A60274B1B889BB2013B94
:105748009AB2254B1A80244B1B889BB2002B19D088
:105758001E4B1B681B78DBB23B601C4B1B6801337C
:105768001A4A1360194B1A68194B1B689A4202D1DE
:10577800164B184A1A60184B1B889BB2013B9AB209
:10578800154B1A803B681A067B681B041A43BB68D2
:105798001B021A43FB6813433B613A697B691A6031
:1057A8000D4B1B889BB2002B7FF46FAF00BF064BDD
:1057B8001B68402BFBD100BF1C37BD465DF8047B3E
:1057C800704700BF0020005038090050D004002066
:1057D800580400209C3801207038012080B584B01E
:1057E80000AF0346FB714E4B1B78002B00F09380F3
:1057F8004C4B1A684C4B1B689A4209D94A4B1B6898
:105808001A46484B1B68D31A03F5AF53FB6006E0F2
:10581800454B1B681A46434B1B68D31AFB60FB6851
:1058280041F2CC5293425FD91920FBF711F83D4B56
:105838001A683D4B1B689A4209D93B4B1B681A46AC
:10584800384B1B68D31A03F5AF53FB6006E0364BA1
:105858001B681A46334B1B68D31AFB60FB6841F27E
:10586800CC52934240D9314BDB68B3F5C06F35D089
:105878005520FBF7B5FF5320FBF7B2FF4220FBF79B
:10588800AFFF5F20FBF7ACFF5420FBF7A9FF7820A0
:10589800FBF7A6FF5F20FBF7A3FF4F20FBF7A0FF56
:1058A8007620FBF79DFF6520FBF79AFF7220FBF738
:1058B80097FF6620FBF794FF6C20FBF791FF6F20A2
:1058C800FBF78EFF7720FBF78BFF2020FBF788FF85
:1058D8002020FBF785FF2020FBF782FF124B144A9C
:1058E8001A60104B124A1A604320FEF74DFC0E4B0B
:1058F8001B685A1C0C490A60FA791A700A4B1A6814
:105908000C4B1B689A4202D1074B094A1A60432084
:10591800FEF720FC00E000BF1037BD4680BD00BF89
:1059280077380120D0040020CC040020004C00402F
:105938009C3801205804002080B582B000AFFAF7E7
:10594800D1FF334B1B78002B01D100235BE0314B97
:105958001A68314B1B689A4254D02E4B1B685A1C4C
:105968002C490A601B78DBB29BB26FEA43436FEAAB
:1059780053437B80274B1A68284B1B689A4202D1F5
:10598800244B274A1A60274B1B78002B09D07B88A9
:1059980048F2F80293420BD07B8848F2FE02934209
:1059A80006D0214B4FF480229A61204BC8221A80DE
:1059B800184B1A68184B1B689A4209D9164B1B6872
:1059C8001A46144B1B68D31A03F5AF537B6006E0E5
:1059D800114B1B681A460F4B1B68D31A7B607B68F8
:1059E80041F2DB4293420BD8114B00221A700E4B46
:1059F80008229A610F4A0F4B1B6843F00443136057
:105A08007B8800E0002318460837BD4680BD00BFEC
:105A180077380120D8040020D40400205C0400203A
:105A28008C4E0120824E012000080048CE1A00202A
:105A3800844E0120400B005080B584B000AF03466F
:105A4800FB71A74B1B780133DAB2A54B1A7097F993
:105A58000730002B80F2E780FB79F72B02D0A04BB0
:105A680001221A70FB79F02B0FD19E4BF0221A708D
:105A78009D4BFF221A709D4B00221A709C4B0022EE
:105A88001A709C4B00221A700BE2FB79F72B40F03E
:105A98008780934B1B78012B35D1974B05221A70C1
:105AA800904BF7221A70954B00221A70944B0022E3
:105AB8001A708D4B00221A708C4B00221A708C4B76
:105AC80000221A708B4B1B78002B0CD0854BF722C9
:105AD8001A708A4B00221A70894B00221A70854B63
:105AE80000221A707FE1804B00221A707C4B002242
:105AF8001A707E4B00221A707D4B00221A707D4B63
:105B080000221A70CDE1764B1B78022B21D17A4BFB
:105B180006221A70734B1B78F02B03D0774B1A7838
:105B2800704B1A70754B1A786E4B1A70734BF722BC
:105B38001A70734B00221A706B4B00221A706B4B51
:105B480000221A706A4B00221A706A4B00221A70DF
:105B580049E1694B07221A70624B1B78F02B07D179
:105B6800644B1B78002B03D1654BF7221A700AE0AF
:105B7800624B1A785B4B1A70614B1A785F4B1A703C
:105B88005F4BF7221A70584B00221A70574B0022AD
:105B98001A70574B00221A70564B00221A7022E1D5
:105BA800504AFB7913704F4B1B78F32B0CD84E4B94
:105BB800FF221A704D4B00221A704D4B00221A70AA
:105BC8004C4B00221A706CE1464B1B78F42B07D023
:105BD800444B1B78F52B03D0424B1B78FD2B0CD183
:105BE800414B00221A70414B00221A70404B002290
:105BF8001A70404B00221A7053E13F4B05221A706D
:105C08003E4B00221A703E4B00221A70364B00227F
:105C18001A70364B00221A70354B00221A70354B19
:105C280000221A70DFE02F4B1B7823F00F03FB7262
:105C38002D4B1B78002B15D12C4B00221A702C4BA6
:105C480000221A702B4B00221A702B4B0F221A704D
:105C5800244AFB791370294B00221A70284B002222
:105C68001A70C0E0214B1B78002B4BD1234AFB79DB
:105C78001370234B00221A701A4B1B78F12B03D098
:105C8800184B1B78F32B0FD11B4B02221A70164BA3
:105C980000221A70154B00221A70154B00221A7038
:105CA800144B00221A709EE0FB7AC02B02D0FB7ABC
:105CB800D02B11D1FB7A1B09DAB20F4B1A700A4BA1
:105CC800FF221A70094B00221A70094B00221A7021
:105CD800084B00221A7086E0044BFF221A70E0E09D
:105CE800814E01207C4E01207D4E01207A38012012
:105CF8007F4E0120834E012076380120804E0120FE
:105D080084380120684B1B78002B0CD1674B00228C
:105D18001A70674B00221A70664B00221A70664B85
:105D280000221A70BDE0634B1B78002B41D1634AF7
:105D3800FB791370604B1B78002B03D05D4BFF225F
:105D48001A70AEE05E4B1B78F22B0FD15D4B03222D
:105D58001A70554B00221A70554B00221A70554B79
:105D680000221A70544B00221A703CE0544B1B78E6
:105D7800F02B0FD1534B04221A704F4BFF221A708D
:105D8800494BFF221A704A4B00221A70494B0022D5
:105D98001A7028E0FB7A1B09DAB24A4B1A70424B98
:105DA800FF221A70424B00221A70424B00221A70CE
:105DB80019E0454B1A78424B1A70404B1A78424BFF
:105DC8001A703E4AFB7913703E4B04221A703A4B04
:105DD800FF221A70344BFF221A70354B00221A70BA
:105DE800344B00221A70394B1B78002B58D04320B3
:105DF800FEF7CAF9364B1B68FB60FB685A1CFA6051
:105E0800304A12781A70334B1B68FA689A4201D1EB
:105E1800314BFB60FB685A1CFA60294A12781A70E9
:105E28002C4B1B68FA689A4201D12B4BFB60FB682C
:105E38005A1CFA60244A12781A70264B1B68FA68B2
:105E48009A4201D1244BFB60FB685A1CFA601B4A3A
:105E580012781A701F4B1B68FA689A4201D11E4BC0
:105E6800FB601B4AFB6813604320FEF773F90F4B76
:105E780000221A700E4B00221A700E4B00221A7064
:105E8800104B1B78072B03D80E4B1B78042B03D120
:105E98000B4B1B78F02B04D9034B00221A7000E03F
:105EA80000BF1037BD4680BD7D4E0120814E0120C8
:105EB8007A3801207F4E0120834E0120843801204A
:105EC8007C4E012076380120804E01207738012051
:105ED800CC040020580400209C380120B0B5A8B09C
:105EE80000AF0346FB71CD4B07F17C041D460FCD77
:105EF8000FC495E80F0007C42370C94B07F1540479
:105F08001D460FCD0FC40FCD0FC495E803002060C8
:105F18000434218002340B0C2370C24B07F1440473
:105F28000FCB07C42370C04B07F134040FCB07C451
:105F38002380BE4B07F10C041D460FCD0FC40FCDB7
:105F48000FC495E80300206004342170FB79602BAE
:105F580005D9FB797A2B02D8FB79203BFB71FB79B9
:105F68000D2B02D0FB790A2B02D1012300F063BC70
:105F7800FB79213B5B2B00F25D8401A252F823F0F0
:105F8800F96000083D6800083D6800083D680008A1
:105F98003D6800083D6800083D6800083D68000845
:105FA8003D6800083D6800083D6800083D68000835
:105FB8003D6800083D6800083D6800083D68000825
:105FC800E16400083D68000837650008E1650008DD
:105FD800376600083D6800083D6800083D6800080D
:105FE8003D6800083D6800083D6800083D680008F5
:105FF8003D6800083D680008396700084D670008DB
:1060080007610008636400083D6800085D620008D5
:106018003D6800084B6300082D610008E561000831
:10602800896100087163000897630008BD63000870
:10603800B7610008896400083D680008E363000848
:106048003D6800080B6300085B610008CB6200082C
:106058009D620008AF6400083D68000823640008DA
:106068008D660008E36600083D6800083D68000882
:106078003D6800083D6800083D6800083D68000864
:106088003D6800083D6800083D6800083D68000854
:106098003D6800083D6800083D6800083D68000844
:1060A8003D6800083D6800083D6800083D68000834
:1060B8003D6800083D6800083D6800083D68000824
:1060C8003D6800083D6800083D6800083D68000814
:1060D8003D6800083D6800083D6800083D68000804
:1060E8003D6800083D6800083D680008B967000879
:1060F80001F012FA0D20FBF715FC01239BE34C4835
:10610800FBF74AFC4B48FBF747FC3A20FBF70AFC35
:106118002020FBF707FC00F081FD0D20FBF702FCB7
:10612800012388E34248FBF737FC4348FBF734FC7C
:106138003A20FBF7F7FB2020FBF7F4FB00F0D6FD35
:106148003E4B1B683E4A13610D20FBF7EBFB012316
:1061580071E33748FBF720FC3A48FBF71DFC3A206F
:10616800FBF7E0FB2020FBF7DDFB00F0BFFD334B26
:106178001B68334A93610D20FBF7D4FB01235AE3D4
:106188002B48FBF709FC3048FBF706FC3A20FBF7E5
:10619800C9FB2020FBF7C6FB00F0A8FD274B1B68B6
:1061A800274A53610D20FBF7BDFB012343E3204839
:1061B800FBF7F2FB2548FBF7EFFB3A20FBF7B2FBB6
:1061C8002020FBF7AFFB00F091FD1C4B1B681C4A1D
:1061D80093620D20FBF7A6FB01232CE31448FBF781
:1061E800DBFB1B48FBF7D8FB3A20FBF79BFB202087
:1061F800FBF798FB4FF6FF7000F000FCC7F89C0017
:10620800D7F89C30B3F5803F03D20D4AD7F89C30BD
:1062180013630D20FBF786FB01230CE3EC8B0008CE
:106228000C8C0008348C0008448C0008548C00083E
:106238007C8E0008A48E0008D08E000870640120AF
:106248007C5C0020188F0008F08E0008448F00083E
:10625800B08F0008CB48FBF79FFBCB48FBF79CFBB4
:106268003A20FBF75FFB2020FBF75CFB4FF6FF7043
:1062780000F0C4FBC7F89C00D7F89C30B3F5803F0A
:1062880003D2C24AD7F89C30D3620D20FBF74AFBF1
:106298000123D0E2BB48FBF77FFBBD48FBF77CFB43
:1062A8003A20FBF73FFB2020FBF73CFB00F01EFDEC
:1062B800B84B1B68B54AD3610D20FBF733FB0123AC
:1062C800B9E2B048FBF768FBB348FBF765FB3A2037
:1062D800FBF728FB2020FBF725FB4FF6FF7000F0AB
:1062E8008DFBC7F89C00D7F89C30B3F5803F03D2EC
:1062F800A64AD7F89C3013620D20FBF713FB012345
:1063080099E2A048FBF748FBA448FBF745FB3A2075
:10631800FBF708FB2020FBF705FB4FF6FF7000F0AA
:106328006DFBC7F89C00D7F89C30B3F5803F03D2CB
:10633800964AD7F89C3053620D20FBF7F3FA0123F5
:1063480079E29048FBF728FB9548FBF725FB3A20B4
:10635800FBF7E8FA2020FBF7E5FA00F087FD0D20AF
:10636800FBF7E0FA012366E28648FBF715FB8D4848
:10637800FBF712FB3A20FBF7D5FA2020FBF7D2FAFD
:1063880000F020FD0D20FBF7CDFA012353E27D48F4
:10639800FBF702FB8448FBF7FFFA3A20FBF7C2FA47
:1063A8002020FBF7BFFA00F037FD0D20FBF7BAFA03
:1063B800012340E27348FBF7EFFA7C48FBF7ECFA5D
:1063C8003A20FBF7AFFA2020FBF7ACFA00F0DAFC32
:1063D8000D20FBF7A7FA01232DE26A48FBF7DCFA48
:1063E8007348FBF7D9FA3A20FBF79CFA2020FBF711
:1063F80099FA4FF6FF7000F001FBC7F89C00D7F838
:106408009C30B3F5803F03D2604AD7F89C30536480
:106418000D20FBF787FA01230DE25A48FBF7BCFA77
:106428006448FBF7B9FA3A20FBF77CFA2020FBF71F
:1064380079FA4FF6FF7000F0E1FAC7F89C00D7F838
:106448009C30B3F5803F03D2504AD7F89C30936410
:106458000D20FBF767FA0123EDE14A48FBF79CFAA8
:106468005548FBF799FA3A20FBF75CFA2020FBF72E
:1064780059FA00F037FD0D20FBF754FA0123DAE151
:106488004048FBF789FA4D48FBF786FA3A20FBF7B4
:1064980049FA2020FBF746FA00F06AFD0D20FBF7C9
:1064A80041FA0123C7E13748FBF776FA4448FBF77E
:1064B80073FA3A20FBF736FA2020FBF733FA00F09C
:1064C8002FFB0346002B02D13F20FBF72BFA0D20B0
:1064D800FBF728FA0123AEE12A48FBF75DFA3948B1
:1064E800FBF75AFA3A20FBF71DFA2020FBF71AFAB5
:1064F80000F034FA0346002B11D0244B9B6B9BB25F
:10650800224A9363214B9B6B2F4A12881204134330
:106518001E4A93632C4B1A882C4B1A8002E03F20AA
:10652800FBF700FA0D20FBF7FDF9012383E115487D
:10653800FBF732FA2648FBF72FFA3A20FBF7F2F975
:106548002020FBF7EFF900F009FA0346002B11D0E1
:106558000E4B9B6B1B0C1B040C4A93630B4B9B6BE6
:10656800194A12881343094A9363174B1A88194B1F
:106578001A8002E03F20FBF7D5F90D20FBF7D2F98E
:10658800012358E17C8E0008748F00087C5C002091
:10659800F48F0008706401206490000830900008AF
:1065A80044910008CC9000080891000888900008E1
:1065B800C0920008009300084493000888930008DC
:1065C800808E0008849100086C64012052380120F4
:1065D800B891000884F600209948FBF7DDF999483E
:1065E800FBF7DAF93A20FBF79DF92020FBF79AF937
:1065F80000F0B4F90346002B11D0934BDB6B9BB230
:10660800914AD363904BDB6B904A12881204134370
:106618008D4AD3638D4B1A888D4B1A8002E03F2038
:10662800FBF780F90D20FBF77DF9012303E184488E
:10663800FBF7B2F98748FBF7AFF93A20FBF772F995
:106648002020FBF76FF900F089F90346002B11D0E1
:106658007D4BDB6B1B0C1B047B4AD3637A4BDB6BD8
:106668007A4A12881343784AD363784B1A887A4B4C
:106678001A8002E03F20FBF755F90D20FBF752F98D
:106688000123D8E06E48FBF787F97448FBF784F9D3
:106698003A20FBF747F92020FBF744F900F05EF9B0
:1066A8000346002B11D0684B1B6C9BB2664A1364DF
:1066B800654B1B6C654A128812041343624A1364C3
:1066C800624B1A88664B1A8002E03F20FBF72AF9D2
:1066D8000D20FBF727F90123ADE05948FBF75CF9DA
:1066E8006048FBF759F93A20FBF71CF92020FBF723
:1066F80019F900F033F90346002B11D0524B1B6CEB
:106708001B0C1B04504A13644F4B1B6C4F4A1288D6
:1067180013434D4A13644D4B1A88534B1A8002E0B9
:106728003F20FBF7FFF80D20FBF7FCF8012382E080
:106738000D20FBF7F7F800F061FC0D20FBF7F2F8ED
:10674800012378E04FF49670FAF782F8FBF762FBC2
:106758000346002B05D03F20FBF7E4F82020FBF789
:10676800E1F807F154031846FBF716F9FBF752FB5B
:106778000346A7F89A30B7F89A30002BF6D0B7F846
:106788009A3048F2400293420BD1FAF73BFA2020A4
:10679800FBF7C8F86F20FBF7C5F86B20FBF7C2F8CA
:1067A80004E007F134031846FBF7F6F8012342E04A
:1067B8004FF49670FAF74CF8FBF72CFB0346002BC6
:1067C80005D03F20FBF7AEF82020FBF7ABF807F128
:1067D8007C031846FBF7E0F8FBF71CFB0346A7F819
:1067E8009A30B7F89A30002BF6D0B7F89A3048F2BA
:1067F8007C02934217D1FAF73BFB0346002B0CD0DF
:106808002020FBF78FF86F20FBF78CF86B20FBF745
:1068180089F80D20FBF786F80AE007F10C03184603
:10682800FBF7BAF804E007F144031846FBF7B4F89D
:10683800012300E000231846A037BD46B0BD00BFC5
:106848007C8E0008EC9100087C5C00206C640120C0
:10685800B4B40020209200084C380120549200085B
:106868005C2201208C9200086838012080B582B033
:1068780000AFFBF7CFFA03467B807B88002BF8D06C
:106888007B88DBB27B607B680A2B05D07B680D2B8D
:1068980002D07B682E2B02D16FF0010326E07B68C3
:1068A8002F2B0AD97B68392B07D87B68DBB21846AF
:1068B800FBF738F87B68303B18E07B68602B05D91C
:1068C8007B687A2B02D87B68203B7B607B68402BF7
:1068D8000AD97B68462B07D87B68DBB21846FBF7DA
:1068E80021F87B68373B01E04FF0FF331846083743
:1068F800BD4680BD80B582B000AFFFF7B7FF7860B6
:106908007B6813F1020F02D14FF0FF3321E07B685F
:106918000F2B02D94FF0FF331BE0FFF7A7FF3860BA
:106928003B6813F1020F01D17B6812E03B680F2B23
:1069380002D94FF0FF330CE0FFF798FF034613F13D
:10694800020F02D04FF0FF3303E07B681A013B6867
:10695800134318460837BD4680BD00BF80B582B0D6
:1069680000AFFFF783FF78607B68FF2B01D9002316
:106978003DE07B689AB2204B1A80FFF777FF78607A
:106988007B68FF2B01D9002331E01B4B1B881B01BF
:106998009AB27B689BB213449AB2174B1A80FFF7DE
:1069A80065FF78607B68FF2B01D900231FE0124B3D
:1069B8001B881B019AB27B689BB213449AB20E4B98
:1069C8001A80FFF753FF78607B68FF2B01D90023FB
:1069D8000DE0094B1B881B019AB27B689BB21344DC
:1069E8009AB2054B1A802020FAF79CFF012318461B
:1069F8000837BD4680BD00BF6C64012080B584B0F7
:106A080000AF78607B68264A934202D94FF0FF3383
:106A180041E00023FB6039E0FBF7FCF903467B818A
:106A28007B89002BF8D07B897B727B7A0A2B05D077
:106A38007B7A0D2B02D07B7A2E2B01D1FB682AE0C2
:106A48007B7A2F2B02D97B7A392B05D93F20FAF78D
:106A580069FF4FF0FF331EE07B7A1846FAF762FFB2
:106A68007B7A303B7B72FA6813469B0013445B00C9
:106A78001A467B7A1344FB60FA687B689A4205D908
:106A88003F20FAF74FFF4FF0FF3304E0FA687B68C6
:106A98009A42C1D9FB6818461037BD4680BD00BF71
:106AA800B782010080B582B000AF78607B68632B45
:106AB80002D83020FAF736FF7B68092B02D830203D
:106AC800FAF730FF7868FBF765F800BF0837BD466E
:106AD80080BD00BF80B582B000AF78607868FBF7F2
:106AE8008BF97B6842F20F72934202D82020FAF7A2
:106AF80019FF7B68B3F57A7F02D22020FAF712FFDC
:106B08007B68632B02D82020FAF70CFF7B68092BDF
:106B180002D82020FAF706FF00BF0837BD4680BD1F
:106B280080B586B000AF3A4A07F10C0392E803003B
:106B3800186004331970374A3B1D92E80300186047
:106B48000433197007F10C031846FAF725FFFFF70D
:106B58008DFE0346FB75FB7DBB82FFF787FE034670
:106B6800FB75BB8A1B019AB2FB7D9BB21344BB82A7
:106B7800FFF77CFE0346FB75BB8A1B019AB2FB7DBF
:106B88009BB21344BB82FFF771FE0346FB75BB8AB9
:106B98001B019AB2FB7D9BB21344BB822020FAF7FB
:106BA800C1FE3B1D1846FAF7F7FEFFF75FFE0346E6
:106BB800FB75FB7D7B82FFF759FE0346FB757B8ADD
:106BC8001B019AB2FB7D9BB213447B82FFF74EFEFA
:106BD8000346FB757B8A1B019AB2FB7D9BB213446B
:106BE8007B82FFF743FE0346FB757B8A1B019AB243
:106BF800FB7D9BB213447B82BB8A074A13607B8A66
:106C0800054A5360012318461837BD4680BD00BFAA
:106C18007C8C0008848C00087C5C002080B584B0E3
:106C280000AFFFF767FEF860FB68FF2B01D9002370
:106C380055E0FB68BB602E20FAF774FEFFF75AFE9A
:106C4800F860FB68FF2B01D9002348E0BB681A02F3
:106C5800FB681343BB602E20FAF764FEFFF74AFE79
:106C6800F860FB68FF2B01D9002338E0FB687B60E4
:106C78002E20FAF757FEFFF73DFEF860FB68FF2B62
:106C880001D900232BE07B681A02FB6813437B6061
:106C98002E20FAF747FEFFF72DFEF860FB68FF2B62
:106CA80001D900231BE07B681A02FB6813437B6051
:106CB8002E20FAF737FEFFF71DFEF860FB68FF2B62
:106CC80001D900230BE07B681A02FB6813437B6041
:106CD800054ABB689360044A7B68D3600123184661
:106CE8001037BD4680BD00BF7C5C002080B582B0F7
:106CF80000AFFF20FFF782FE78607B68FF2B01D989
:106D0800002338E07B683B602E20FAF70BFEFF205B
:106D1800FFF774FE78607B68FF2B01D900232AE017
:106D28003B681A027B6813433B602E20FAF7FAFD92
:106D3800FF20FFF763FE78607B68FF2B01D90023F3
:106D480019E03B681A027B6813433B602E20FAF770
:106D5800E9FDFF20FFF752FE78607B68FF2B01D921
:106D6800002308E03B681A027B6813433B60044A2F
:106D78003B681360012318460837BD4680BD00BF35
:106D88007064012080B582B000AF0220FFF736FEA4
:106D980078607B68022B03D93F20FAF7C3FD0BE02C
:106DA800074B5B6B23F00F03054A5363044B5A6B85
:106DB8007B681343024A53630837BD4680BD00BF52
:106DC8007C5C002080B582B000AF0120FFF716FE82
:106DD80078607B68012B03D93F20FAF7A3FD13E005
:106DE8007B68DBB203F00103DAB2094B1A70094B76
:106DF8005B6B23F0F003074A5363064B5A6B7B68BF
:106E08001B011343034A53630837BD4680BD00BFC7
:106E1800A1E000207C5C002080B582B000AF01209A
:106E2800FFF7ECFD78607B68012B03D93F20FAF768
:106E380079FD13E07B68DBB203F00103DAB2094B9A
:106E48001A70094B5B6B23F47063074A5363064B54
:106E58005A6B7B681B021343034A53630837BD46CA
:106E680080BD00BF6A3801207C5C002080B582B0FC
:106E780000AF0720FFF7C2FD78607B68072B03D9B6
:106E88003F20FAF74FFD21E07B68DBB203F00403F3
:106E9800DAB2104B1A707B68DBB203F00203DAB285
:106EA8000D4B1A707B68DBB203F00103DAB20B4BAF
:106EB8001A700B4B5B6B23F47043094A5363084BFE
:106EC8005A6B7B681B031343054A53630837BD4657
:106ED80080BD00BF9DE000205922012042380120DA
:106EE8007C5C002080B582B000AF6020FFF786FD93
:106EF80078607B68602B03D93F20FAF713FD32E0F6
:106F08007B681F2B1BD01F2B06D8132B0FD0172BDA
:106F180011D00B2B07D022E0392B18D0602B1AD0B8
:106F2800262B10D01BE0114A7B68D3641BE00F4A64
:106F38007B68D36417E00D4A7B68D36413E00B4A7F
:106F48007B68D3640FE0094A7B68D3640BE0074A87
:106F58007B68D36407E0054A7B68D36403E03F207D
:106F6800FAF7E0FC00BF0837BD4680BD7C5C002016
:106F780080B582B000AF6020FFF740FD78607B6885
:106F8800602B03D93F20FAF7CDFC32E07B681F2B3A
:106F98001BD01F2B06D8132B0FD0172B11D00B2B60
:106FA80007D022E0392B18D0602B1AD0262B10D00E
:106FB8001BE0114A7B6813651BE00F4A7B68136569
:106FC80017E00D4A7B68136513E00B4A7B6813656D
:106FD8000FE0094A7B6813650BE0074A7B68136575
:106FE80007E0054A7B68136503E03F20FAF79AFC3F
:106FF80000BF0837BD4680BD7C5C0020B0B5B8B086
:1070080000AFE14B07F1C8041D460FCD0FC495E84A
:10701800030084E80300DD4B07F1B4041D460FCDDF
:107028000FC42B682380DA4A07F170031146412206
:10703800184601F0B7FDD74A07F12C031146442240
:10704800184601F0AFFDD44B07F11C040FCB07C461
:107058002380D24B3C1D1D460FCD0FC495E803007D
:107068002060043421700D20FAF75CFC07F11C0342
:107078001846FAF791FC3120FAF754FC2E20FAF75B
:1070880051FC3720FAF74EFC3B1D1846FAF784FCF2
:107098000D20FAF747FC07F1C8031846FAF77CFCFD
:1070A8000D20FAF73FFC2120FAF73CFC3A20FAF7CA
:1070B80039FC2020FAF736FC07F1B4031846FAF732
:1070C8006BFC0D20FAF72EFC5620FAF72BFC3A2021
:1070D800FAF728FC2020FAF725FCB148FAF75CFCFF
:1070E800B048FAF759FC0D20FAF71CFC4120FAF7D2
:1070F80019FC3A20FAF716FC2020FAF713FCA848E6
:10710800FAF74AFCA848FAF747FC0D20FAF70AFCF8
:107118004720FAF707FC3A20FAF704FC2020FAF790
:1071280001FC9F48FAF738FCA048FAF735FC0D2017
:10713800FAF7F8FB4920FAF7F5FB3A20FAF7F2FBE1
:107148002020FAF7EFFB9648FAF726FC9848FAF75A
:1071580023FC0D20FAF7E6FB5320FAF7E3FB3A206D
:10716800FAF7E0FB2020FAF7DDFB8D48FAF714FC6C
:107178009048FAF711FC0D20FAF7D4FB4D20FAF7E6
:10718800D1FB3A20FAF7CEFB2020FAF7CBFB844854
:10719800FAF702FC8848FAF7FFFB0D20FAF7C2FB62
:1071A8004820FAF7BFFB3A20FAF7BCFB2020FAF791
:1071B800B9FB7B48FAF7F0FB8048FAF7EDFB0D20A6
:1071C800FAF7B0FB4420FAF7ADFB3A20FAF7AAFB2E
:1071D8002020FAF7A7FB7248FAF7DEFB7848FAF79F
:1071E800DBFB0D20FAF79EFB5520FAF79BFB3A20B4
:1071F800FAF798FB2020FAF795FB6948FAF7CCFBD9
:107208007048FAF7C9FB0D20FAF78CFB5220FAF701
:1072180089FB3A20FAF786FB2020FAF783FB6048BF
:10722800FAF7BAFB6848FAF7B7FB0D20FAF77AFBCA
:107238005420FAF777FB3A20FAF774FB2020FAF784
:1072480071FB5748FAF7A8FB6048FAF7A5FB0D2031
:10725800FAF768FB4C20FAF765FB3A20FAF762FB6D
:107268002020FAF75FFB4E48FAF796FB5848FAF7E2
:1072780093FB0D20FAF756FB5020FAF753FB3A2000
:10728800FAF750FB2020FAF74DFB4548FAF784FB44
:107298005048FAF781FB0D20FAF744FB5820FAF71B
:1072A80041FB3A20FAF73EFB2020FAF73BFB3C482B
:1072B800FAF772FB4848FAF76FFB0D20FAF732FB32
:1072C8004220FAF72FFB3A20FAF72CFB2020FAF796
:1072D80029FB3348FAF760FB4048FAF75DFB0D20BD
:1072E800FAF720FB4E20FAF71DFB3A20FAF71AFBB3
:1072F8002020FAF717FB2A48FAF74EFB3848FAF726
:107308004BFB0D20FAF70EFB4A20FAF70BFB3A204D
:10731800FAF708FB2020FAF705FB2148FAF73CFBAF
:107328003048FAF739FB0D20FAF7FCFA4B20FAF748
:10733800F9FA3A20FAF7F6FA2020FAF7F3FA184899
:10734800FAF72AFB2848FAF727FB0D20FAF7EAFA9A
:107358004620FAF7E7FA3A20FAF7E4FA2020FAF793
:10736800E1FA0F48FAF718FB2048FAF715FB0D2049
:10737800FAF7D8FA3120FAF7D5FA3A20FAF7D2FA1A
:107388002020FAF7CFFA33E08C8C0008A48C000890
:10739800B88C0008FC8C0008408D0008508D00084F
:1073A8007C8E0008808E0008A48E0008D08E00080D
:1073B800F08E0008188F0008448F0008B08F00086E
:1073C800748F0008F48F000830900008649000085B
:1073D80088900008C09200080093000844930008B1
:1073E80088930008CC900008089100084491000890
:1073F8004248FAF7D1FA4248FAF7CEFA0D20FAF7DE
:1074080091FA3320FAF78EFA3A20FAF78BFA20200D
:10741800FAF788FA3948FAF7BFFA3A48FAF7BCFA9D
:107428000D20FAF77FFA3420FAF77CFA3A20FAF7B7
:1074380079FA2020FAF776FA3048FAF7ADFA3248A6
:10744800FAF7AAFA0D20FAF76DFA3520FAF76AFA70
:107458003A20FAF767FA2020FAF764FA2748FAF789
:107468009BFA2A48FAF798FA0D20FAF75BFA59209E
:10747800FAF758FA3A20FAF755FA2020FAF752FAAA
:107488001E48FAF789FA2248FAF786FA0D20FAF721
:1074980049FA5A20FAF746FA3A20FAF743FA20202E
:1074A800FAF740FA1548FAF777FA1A48FAF774FA29
:1074B8000D20FAF737FA4020FAF734FA3A20FAF7AB
:1074C80031FA2020FAF72EFA07F12C031846FAF7BA
:1074D80063FA0D20FAF726FA7C20FAF723FA3A2005
:1074E800FAF720FA2020FAF71DFA07F17003184678
:1074F800FAF752FA00BFE037BD46B0BD7C8E0008EF
:1075080084910008B8910008EC91000820920008C6
:10751800549200088C920008B0B586B000AFCD4BED
:107528003C461D460FCD0FC495E803002060043487
:1075380021800D20FAF7F6F93B461846FAF72CFA9F
:107548000D20FAF7EFF95620FAF7ECF93A20FAF796
:10755800E9F92020FAF7E6F9BF4B1B689BB21846F9
:10756800FAF788FA2F20FAF7DDF92020FAF7DAF986
:10757800B94B5B689BB21846FAF77CFAB748FAF73A
:107588000BFA0D20FAF7CEF94120FAF7CBF93A2099
:10759800FAF7C8F92020FAF7C5F9AF4B9B681B0A20
:1075A800DBB21846FAF73CFA2E20FAF7BBF9AA4BD9
:1075B8009B68DBB21846FAF733FA2E20FAF7B2F9CD
:1075C800A54BDB681B0EDBB21846FAF729FA2E200A
:1075D800FAF7A8F9A04BDB681B0CDBB21846FAF7E0
:1075E8001FFA2E20FAF79EF99B4BDB681B0ADBB2C9
:1075F8001846FAF715FA2E20FAF794F9964BDB6835
:10760800DBB21846FAF70CFA9548FAF7C5F90D20D7
:10761800FAF788F94720FAF785F93A20FAF782F954
:107628002020FAF77FF98C4B1B691B0E1846FFF7D1
:1076380039FA2E20FAF776F9874B1B691B0CDBB257
:107648001846FFF72FFA2E20FAF76CF9824B1B69C0
:107658001B0ADBB21846FFF725FA2E20FAF762F963
:107668007D4B1B69DBB21846FFF71CFA7D48FAF719
:1076780093F90D20FAF756F94920FAF753F93A2009
:10768800FAF750F92020FAF74DF9734B5B691B0E96
:107698001846FFF707FA2E20FAF744F96E4B5B6994
:1076A8001B0CDBB21846FFF7FDF92E20FAF73AF962
:1076B800694B5B691B0ADBB21846FFF7F3F92E200A
:1076C800FAF730F9644B5B69DBB21846FFF7EAF961
:1076D8006548FAF761F90D20FAF724F95320FAF70B
:1076E80021F93A20FAF71EF92020FAF71BF95A4B2C
:1076F8009B691B0E1846FFF7D5F92E20FAF712F9E9
:10770800554B9B691B0CDBB21846FFF7CBF92E20B3
:10771800FAF708F9504B9B691B0ADBB21846FFF7CA
:10772800C1F92E20FAF7FEF84B4B9B69DBB21846DD
:10773800FFF7B8F94D48FAF72FF90D20FAF7F2F8E4
:107748004D20FAF7EFF83A20FAF7ECF82020FAF78C
:10775800E9F8414B9B6A1B0E1846FFF7A3F92E2048
:10776800FAF7E0F83C4B9B6A1B0CDBB21846FFF7B4
:1077780099F92E20FAF7D6F8374B9B6A1B0ADBB229
:107788001846FFF78FF92E20FAF7CCF8324B9B6A90
:10779800DBB21846FFF786F93548FAF7FDF80D20F1
:1077A800FAF7C0F84820FAF7BDF83A20FAF7BAF81D
:1077B8002020FAF7B7F8284B1B6B9BB21846FFF747
:1077C80089F92C48FAF7E8F80D20FAF7ABF84420C5
:1077D800FAF7A8F83A20FAF7A5F82020FAF7A2F85D
:1077E8001D4BDB6A9BB21846FFF774F92248FAF77B
:1077F800D3F80D20FAF796F85520FAF793F83A20BF
:10780800FAF790F82020FAF78DF8134BDB691B0E76
:107818001846FFF747F92E20FAF784F80E4BDB6974
:107828001B0CDBB21846FFF73DF92E20FAF77AF861
:10783800094BDB691B0ADBB21846FFF733F92E2028
:10784800FAF770F8044BDB69DBB21846FFF72AF940
:1078580014E000BF688D00087C5C0020808E000862
:10786800A48E0008D08E0008F08E0008188F00083B
:10787800448F0008B08F0008748F0008D548FAF7C5
:107888008BF80D20FAF74EF85220FAF74BF83A2009
:10789800FAF748F82020FAF745F8CF4B5B6A9BB215
:1078A8001846FFF717F9CD48FAF776F80D20FAF7DA
:1078B80039F85420FAF736F83A20FAF733F8202046
:1078C800FAF730F8C44B1B6A9BB21846FFF702F967
:1078D800C348FAF761F80D20FAF724F84C20FAF7B4
:1078E80021F83A20FAF71EF82020FAF71BF8BA4BCD
:1078F8005B6B03F00F031846FFF7ECF8B948FAF78B
:107908004BF80D20FAF70EF85020FAF70BF83A204A
:10791800FAF708F82020FAF705F8AF4B5B6C9BB232
:107928001846FFF7D7F8B048FAF736F80D20F9F7F8
:10793800F9FF5820F9F7F6FF3A20F9F7F3FF20206E
:10794800F9F7F0FFA44B9B6C9BB21846FFF7C2F8FF
:10795800A648FAF721F80D20F9F7E4FF4220F9F7D5
:10796800E1FF3A20F9F7DEFF2020F9F7DBFF9A4B19
:10797800DB6C9F4AA2FB0323DB08DBB23033DBB2AC
:107988001846F9F7CFFF944BD96C994BA3FB012309
:10799800DA0813469B0013445B00CA1AD3B230338B
:1079A800DBB21846F9F7BEFF8B4BDB6C1F2B36D0CA
:1079B8001F2B06D8132B18D0172B23D00B2B07D02F
:1079C80061E0392B45D0602B50D0262B34D05AE0BB
:1079D8003520F9F7A7FF3220F9F7A4FF3020F9F78F
:1079E800A1FF3020F9F79EFF59E03220F9F79AFFFE
:1079F8003020F9F797FF3020F9F794FF2020F9F7A6
:107A080091FF4CE03020F9F78DFF3420F9F78AFF19
:107A18003020F9F787FF3020F9F784FF3FE04D2049
:107A2800F9F780FF4920F9F77DFF4420F9F77AFF3D
:107A38004920F9F777FF32E03420F9F773FF302057
:107A4800F9F770FF3020F9F76DFF2020F9F76AFF8A
:107A580025E03620F9F766FF3020F9F763FF30207C
:107A6800F9F760FF2020F9F75DFF18E03020F9F7FB
:107A780059FF3020F9F756FF2020F9F753FF20204F
:107A8800F9F750FF0BE03F20F9F74CFF3F20F9F7DB
:107A980049FF3F20F9F746FF2020F9F743FF5548F3
:107AA800F9F77AFF0D20F9F73DFF4E20F9F73AFF75
:107AB8003A20F9F737FF2020F9F734FF464B1B6DC2
:107AC8004B4AA2FB0323DB08DBB23033DBB2184698
:107AD800F9F728FF404B196D454BA3FB0123DA0842
:107AE80013469B0013445B00CA1AD3B23033DBB28F
:107AF8001846F9F717FF384B1B6D1F2B36D01F2B75
:107B080006D8132B18D0172B23D00B2B07D073E0D4
:107B1800392B45D0602B50D0262B34D06CE0352043
:107B2800F9F700FF3220F9F7FDFE3020F9F7FAFEE9
:107B38003020F9F7F7FE6BE03220F9F7F3FE30203A
:107B4800F9F7F0FE3020F9F7EDFE2020F9F7EAFE0C
:107B58005EE03020F9F7E6FE3420F9F7E3FE302046
:107B6800F9F7E0FE3020F9F7DDFE51E04D20F9F796
:107B7800D9FE4920F9F7D6FE4420F9F7D3FE49206B
:107B8800F9F7D0FE44E03420F9F7CCFE3020F9F7BD
:107B9800C9FE3020F9F7C6FE2020F9F7C3FE37E00A
:107BA8003620F9F7BFFE3020F9F7BCFE3020F9F790
:107BB800B9FE2020F9F7B6FE2AE03020F9F7B2FE28
:107BC8003020F9F7AFFE2020F9F7ACFE2020F9F7B6
:107BD800A9FE1DE0F48F00087C5C002030900008AE
:107BE8006490000888900008C0920008009300087C
:107BF800CDCCCCCC449300083F20F9F793FE3F202E
:107C0800F9F790FE3F20F9F78DFE2020F9F78AFE5C
:107C18006F48F9F7C1FE0D20F9F784FE4A20F9F7FD
:107C280081FE3A20F9F77EFE2020F9F77BFE694BAA
:107C38005B6B1B0903F00F031846FEF74BFF664802
:107C4800F9F7AAFE0D20F9F76DFE4B20F9F76AFE49
:107C58003A20F9F767FE2020F9F764FE5D4B5B6B6D
:107C68001B0A03F00F031846FEF734FF5B48F9F7C9
:107C780093FE0D20F9F756FE4620F9F753FE3A20F9
:107C8800F9F750FE2020F9F74DFE524B5B6B1B0BAA
:107C980003F00F031846FEF71DFF5148F9F77CFE65
:107CA8000D20F9F73FFE3120F9F73CFE3A20F9F7AD
:107CB80039FE2020F9F736FE464B9B6B1B0C9BB216
:107CC8001846F9F7D7FE2020F9F72CFE4548F9F7B2
:107CD80063FE0D20F9F726FE3320F9F723FE3A203C
:107CE800F9F720FE2020F9F71DFE3A4B9B6B9BB25B
:107CF8001846F9F7BFFE2020F9F714FE3A48F9F7BD
:107D08004BFE0D20F9F70EFE3420F9F70BFE3A2052
:107D1800F9F708FE2020F9F705FE2E4BDB6B1B0C4C
:107D28009BB21846F9F7A6FE2020F9F7FBFD2F486D
:107D3800F9F732FE0D20F9F7F5FD3520F9F7F2FDD8
:107D48003A20F9F7EFFD2020F9F7ECFD214BDB6B2A
:107D58009BB21846F9F78EFE2020F9F7E3FD244878
:107D6800F9F71AFE0D20F9F7DDFD5920F9F7DAFDCC
:107D78003A20F9F7D7FD2020F9F7D4FD154B1B6CF5
:107D88001B0C9BB21846F9F775FE2020F9F7CAFDBF
:107D98001848F9F701FE0D20F9F7C4FD5A20F9F744
:107DA800C1FD3A20F9F7BEFD2020F9F7BBFD094BCC
:107DB8001B6C9BB21846F9F75DFE2020F9F7B2FD5F
:107DC8000D48F9F7E9FD00BF1837BD46B0BD00BF43
:107DD800889300087C5C0020CC900008089100087B
:107DE8004491000884910008B8910008EC910008BB
:107DF80020920008549200088C92000880B500AFC9
:107E0800224B4FF480129A610520F8F721FD1F4B91
:107E180010229A616420F8F71BFD6420F8F718FD1A
:107E2800102201211E2000F021FC102201211F2018
:107E380000F01CFC164B9B689BB21A4600210920D7
:107E480000F03EFC124BDB681A4600210B2000F0C4
:107E580081FC0F4B1B691A460021012000F07AFCB7
:107E68000B4B9B691A460021052000F073FC084B58
:107E78005B691A4600210F2000F06CFCFF220121EB
:107E8800022000F0F3FB0123184680BD00080048DB
:107E9800D45C002080B582B000AF474B5B6A9BB2D0
:107EA8001A460121042000F00BFC434B1B6A9BB2CD
:107EB8001A460121102000F003FC3F4BDB691A46EB
:107EC80001210C2000F046FC3B4BDB6903F07043BA
:107ED800B3F1604F3ED1394B82221A704FF4807251
:107EE8000121062000F0ECFB334BDB6923F07F43D4
:107EF80043F0BC431A460121082000F02BFC1E2247
:107F08000121162000F0B2FB2D4B41F288321A8075
:107F180000212E2000F06EFC0346FB71294B4AF627
:107F2800AA221A60264B1B88002B05D0FB7903F088
:107F3800FD03BD2BECD100E000BF6420F8F788FCFE
:107F480082220121002000F091FB4FF47A70F8F7AB
:107F58007FFC07E0194B02221A700222012100203F
:107F680000F084FB01220121012000F07FFB0023A7
:107F7800FB710121032000F03DFC0346FB71FB79F6
:107F8800222BF6D1FF220121022000F06FFB0022F4
:107F980001212C2000F06AFB00220021172000F0AC
:107FA80065FB00220021182000F060FB0123184621
:107FB8000837BD4680BD00BFD45C00207670012024
:107FC800785C00200030004080B582B000AF464B9E
:107FD8001B6B9BB21A460121042000F071FB424B37
:107FE800DB6A9BB21A460121102000F069FB3E4B68
:107FF8009B6A1A4601210C2000F0ACFB3A4B9B6AA5
:1080080003F07043B3F1604F3BD1384B41F28832F3
:108018001A8000212E2000F0EDFB0346FB71344B43
:108028004AF6AA221A60314B1B88002B05D0FB792F
:1080380003F0FD03BD2BECD100E000BF2D4B8222E5
:108048001A704FF480720121062000F039FB264B8C
:108058009B6A23F07F4343F0BC431A460121082062
:1080680000F078FB1E220121162000F0FFFA4FF4E1
:108078007A70F8F7EDFB82220121002000F0F6FA71
:1080880007E01C4B02221A7002220121002000F096
:10809800EDFA01220121012000F0E8FA0121032074
:1080A80000F0A8FB0346FB71FB79222BF6D10220D6
:1080B800F8F7CEFBFF220121022000F0D7FA0022B8
:1080C80001212C2000F0D2FA00220021172000F014
:1080D800CDFA00220021182000F0C8FA0123184622
:1080E8000837BD4680BD00BFD45C0020785C002006
:1080F800003000407670012080B582B000AF0122C8
:108108000121002000F0B2FA184B01221A70184B16
:108118005B6C9BB21A460121042000F0D1FA0122BF
:108128000121012000F0A2FA0023FB7101210320A4
:1081380000F060FB0346FB71FB79132BF6D1F8F7CF
:10814800A3FB02220121012000F090FA0121032063
:1081580000F050FB0346FB71FB79142BF6D100F0BD
:1081680017F8012318460837BD4680BD76700120F0
:10817800D45C002080B500AF08220121012000F066
:1081880075FA024B00221A8000BF80BD747001206E
:1081980080B500AFFF220121022000F067FAFF221C
:1081A80001212C2000F062FA01220021172000F0A2
:1081B8005DFA01220021182000F058FA00BF80BDA6
:1081C80080B584B000AF0346FB71234B1B78012BAD
:1081D8000AD10121032000F00DFB0346FB81FB8936
:1081E800172B01D0002333E00121202000F028FBC9
:1081F8000346FB81FB89002B01D1002328E00121E4
:10820800242000F01DFB0346BB81FA79BB890221BB
:10821800184600F02BFABB890133BB81BB891A468B
:108228000121242000F04CFA20220121012000F035
:108238001DFA094B1B78012B04D1084B9B6C9AB291
:10824800074B1A80FF220121022000F00FFA0123B8
:1082580018461037BD4680BD76700120D45C0020DA
:108268007470012080B584B000AF78600B467B80C5
:108278000121032000F0BEFA0346FB811D4B1B7849
:10828800012B04D1FB89172B01D000232EE00121FB
:10829800202000F0D5FA0346FB81FA897B889A42B0
:1082A80001D2002322E00121242000F0C9FA03466C
:1082B800BB817A88BB897968184600F053FB03466E
:1082C800BB81BB891A460121242000F0F9F920223C
:1082D8000121012000F0CAF9064B1B78012B04D1BB
:1082E800054B9B6C9AB2054B1A8001231846103730
:1082F800BD4680BD76700120D45C002074700120DA
:1083080080B584B000AF0121262000F099FA034619
:10831800FB81FB89002B01D1012335E0FB89082B68
:1083280001D8002330E00121282000F089FA034613
:10833800BB81BB890321184600F0C8FAB860BB8925
:108348000433BB81BB890321184600F0BFFAB8602B
:10835800FB89083BFB81BB890433BB81BB68FB807D
:10836800FA88BB891146184600F06CFB0346BB81AE
:10837800BB891A460121282000F0A2F940220121D8
:10838800012000F073F9012318461037BD4680BD5F
:1083980080B582B000AF0121032000F02BFA03461C
:1083A800FB71FB79172B01D0002329E0012126203E
:1083B80000F046FA0346BB80BB88002B01D101239D
:1083C8001EE00121282000F03BFA03467B80BA8892
:1083D8007B881146184600F035FB03467B807B8876
:1083E8001A460121282000F06BF9402201210120C2
:1083F80000F03CF9044B9B6C9AB2044B1A800123A1
:1084080018460837BD4680BDD45C00207470012032
:1084180080B582B000AFF8F765FA274B1A68274B8A
:108428001B689A4242D0244B1B685A1C22490A6096
:108438001B789BB26FEA43436FEA5343FB801E4BA2
:108448001A681F4B1B689A4202D11B4B1D4A1A60BF
:108458001D4B1B78102B20D9FB8848F2F802934259
:1084680005D11A4B1B78002B01D000231FE0FB8895
:1084780048F2FE02934205D1154B1B78002B01D020
:10848800002314E0FB8848F2F602934205D1114B11
:108498001B78002B01D0002309E00F4B4FF48022FA
:1084A8009A610E4BC8221A80FB8800E00023184608
:1084B8000837BD4680BD00BFE0040020DC04002072
:1084C8006004002078700120D01A00204238012072
:1084D800592201209DE0002000080048CE1A002003
:1084E80080B400AF464A464B1B6E43F48053136674
:1084F800444A444B1B6823F070531360414A414B74
:108508001B6843F0806313603E4A3E4B5B6823F46C
:10851800005353603B4A3B4BDB6823F04053D36026
:10852800384A384BDB6843F08053D360354A354BC3
:108538009B6823F0705323F47C639360314A314B7A
:108548009B6843F0A05343F4A86393602D4B4FF40A
:1085580000529A612C4A2C4B1B6843F480731360B9
:10856800294A294B5B6823F010035360264A264B9F
:108578009B6823F440739360234A234B9B6843F41E
:1085880080739360204B10229A611E4A1D4B1B6812
:1085980023F47C6313601B4A1A4B1B6843F428635B
:1085A8001360184A174B1B6A23F47F0323F47043A4
:1085B8001362144A134B1B6A43F4AA0343F4A043FF
:1085C8001362124B124A1A60124B114A1A60124B6C
:1085D800124A1A60124B114A1A60124B4FF4417238
:1085E8001A60104B4FF470625A600E4A0D4B1B68AC
:1085F80043F04003136000BFBD465DF8047B70473D
:10860800001002400004004800080048DC04002074
:1086180078700120E0040020E40400207464012044
:10862800E80400200030014080B483B000AF034666
:10863800FB8000BF0C4B9B6803F00203002BF9D0B2
:10864800094AFB88D36000BF074B9B6803F001030E
:10865800002BF9D0044BDB689BB218460C37BD469B
:108668005DF8047B704700BF0030014080B584B0DE
:1086780000AF0346FB800B467B7113463B710F4BE3
:108688004FF000529A617B79DB021BB243F480639E
:108698001AB23B791BB213431BB2FB81FB88184605
:1086A800FFF7C2FFFB891846FFF7BEFF034B4FF4E5
:1086B80000529A6100BF1037BD4680BD00040048D3
:1086C80080B584B000AF0346FB800B467B71134630
:1086D8007B801F4B4FF000529A617B79DB029AB284
:1086E8007B881B0A9BB213439BB243F48063FB81D4
:1086F800FB881846FFF798FFFB891846FFF794FF99
:10870800134B4FF400529A617B79DB021BB243F49E
:1087180080631AB2B7F90230DBB21BB213431BB243
:10872800FB810B4B4FF000529A61FB8801339BB2DF
:108738001846FFF779FFFB891846FFF775FF044BCA
:108748004FF400529A6100BF1037BD4680BD00BF8C
:108758000004004880B584B000AF03463A60FB804F
:108768000B467B71224B4FF000529A617B799BB28A
:10877800DB029AB23B681B0E9BB213439BB243F4D5
:108788008063FB81FB881846FFF74EFFFB8918467C
:10879800FFF74AFF164B4FF400529A617B79DB02D0
:1087A8001BB243F480631AB23B681B0C1BB2DBB2EA
:1087B8001BB213431BB2FB810D4B4FF000529A6161
:1087C800FB8801339BB21846FFF72EFFFB8918463A
:1087D800FFF72AFF3B689BB21846FFF725FF044BBB
:1087E8004FF400529A6100BF1037BD4680BD00BFEC
:1087F8000004004880B584B000AF03460A46FB80F9
:1088080013467B710D4B4FF000529A61FB88184656
:10881800FFF70AFF7B799BB2DB02FB81FB891846D5
:10882800FFF702FF0346BB81044B4FF400529A61E5
:10883800BB89DBB218461037BD4680BD000400482E
:1088480080B584B000AF03460A46FB8013467B71AF
:108858001D4B4FF000529A617B799BB2DB02FB8182
:10886800FB881846FFF7E0FEFB891846FFF7DCFE99
:108878000346BB81144B4FF400529A617B799BB23B
:10888800DB02FB81104B4FF000529A61FB880133E9
:108898009BB21846FFF7C8FEFB891846FFF7C4FECF
:1088A80003467B81084B4FF400529A61BB891B0237
:1088B8001AB2B7F90A30DBB21BB213431BB29BB230
:1088C80018461037BD4680BD0004004880B586B004
:1088D80000AF03460A46FB8013467B71204B4FF0DE
:1088E80000529A617B799BB2DB02FB82FB881846B7
:1088F800FFF79AFEFB8A1846FFF796FE03463B6190
:10890800174B4FF400529A617B799BB2DB02FB82D2
:10891800134B4FF000529A61FB8801339BB2184603
:10892800FFF782FEFB8A1846FFF77EFE0346FB60D0
:108938000020FFF779FE0346BB60094B4FF4005255
:108948009A613B691A06FB681B0403F47F031A4308
:10895800BB689BB2134318461837BD4680BD00BF9D
:108968000004004880B584B000AF03463960FB803E
:108978001346BB80324B4FF000529A61BB8803F01C
:108988000103002B15D13B685A1C3A601B789BB237
:1089980043F4A053FB81FB881846FFF745FEFB898B
:1089A8001846FFF741FEBB88013BBB80FB880133BB
:1089B800FB80234B4FF400529A613B685A1C3A6083
:1089C8001B789BB243F4A053FB811D4B4FF0005220
:1089D8009A61FB881846FFF727FEFB891846FFF7C0
:1089E80023FEBB88013BBB80FB880133FB801AE078
:1089F8003B685A1C3A601B787B733B685A1C3A6088
:108A08001B783B737B7B1B021AB23B7B1BB2134365
:108A18001BB29BB21846FFF707FEBB88023BBB8020
:108A2800FB880233FB80BB88002BE1D1044B4FF459
:108A380000529A61FB8818461037BD4680BD00BFBA
:108A48000004004880B584B000AF03460A46FB80A6
:108A58001346BB804F4B4FF000529A61BB8803F01E
:108A68000103002B25D14FF4C053FB81FB88184626
:108A7800FFF7DAFDFB891846FFF7D6FD0346BB81F1
:108A8800454B1B68BA89D2B21A70434B1B68013335
:108A9800414A1360404B1A68404B1B689A4202D304
:108AA8003D4B3F4A1A60BB88013BBB80FB880133C2
:108AB800FB80384B4FF400529A614FF4C053FB814E
:108AC8004FF4C053FB81334B4FF000529A61FB883F
:108AD8001846FFF7A9FDFB891846FFF7A5FD0346D1
:108AE800BB812D4B1B68BA89D2B21A702A4B1B68FE
:108AF8000133294A1360284B1A68284B1B689A428D
:108B080002D3254B264A1A60BB88013BBB80FB88F1
:108B18000133FB8032E00020FFF786FD0346BB816E
:108B28001D4B1B68BA89120A92B2D2B21A701A4B3C
:108B38001B680133184A1360174B1A68174B1B68D8
:108B48009A4202D3144B164A1A60134B1B68BA890F
:108B5800D2B21A70104B1B6801330F4A13600E4BC8
:108B68001A680E4B1B689A4202D30B4B0C4A1A60C8
:108B7800BB88023BBB80FB880233FB80BB88002B91
:108B8800C9D1044B4FF400529A61FB88184610373C
:108B9800BD4680BD00040048DC04002060040020BD
:108BA8007870012010B5431E0A44914204D011F890
:108BB800014B03F8014FF8E710BD0000F8B500BFFE
:108BC800F8BC08BC9E467047F8B500BFF8BC08BCA6
:048BD8009E467047FE
:108BDC0020464C415348204552524F522021000010
:108BEC005361766520746F20466C6173683F2D3E2F
:108BFC00707265737320616761696E2000000000FC
:108C0C0052656C6F61642053657475702066726F69
:108C1C006D20466C6173683F2D3E707265737320D6
:108C2C00616761696E200000204E4F5420534156FD
:108C3C004544212000000000204E4F54204C4F4151
:108C4C00444544212000000020466C617368205785
:108C5C0072697465204572726F722C20646F205398
:108C6C006574757020616761696E212000000000D9
:108C7C005669643D000000005069643D000000002E
:108C8C004C697374206F6620536574757020436F44
:108C9C006D6D616E64733A0073686F772041637415
:108CAC0075616C2053657475700000007361766596
:108CBC00206E6577207365747570207065726D61B8
:108CCC006E656E746C79202877696C6C20626563B4
:108CDC006F6D6520616374697665206174206E65C3
:108CEC00787420506F776572205570290000000051
:108CFC0072656C6F61642073657475702066726F39
:108D0C006D20466C61736820286368616E676573BB
:108D1C002073696E6365206C61737420506F776586
:108D2C0072205570206172652063616E63656C6C96
:108D3C00656429004D696469204D65726765722010
:108D4C0076000000202863293230313720572E530B
:108D5C006368656D6D657274000000004C69737416
:108D6C00206F662041637475616C20536574757057
:108D7C003A00000043000000000000201201000235
:108D8C00020000408304405707010000000100006E
:108D9C000902430002010080630904000001020281
:108DAC00000005240010010524010300042402071F
:108DBC000524060001070583031000400904010087
:108DCC00020A0000000705810240000107050202AB
:108DDC004000010018034D004900440049002000E8
:108DEC004D006500720067006500720000C2010052
:108DFC0000000800120100020000004083044058EB
:108E0C000701000100010000090265000201008059
:108E1C00630904000000010100000924010001099C
:108E2C0000010109040100020103000007240100F4
:108E3C00014100062402010100062402020200097D
:108E4C0024030103010201000924030204010101AE
:108E5C0000090581024000000000052501010309FD
:108E6C000502024000000000052501010100000080
:108E7C007365740020555342205669642F50696401
:108E8C00206F662074686973206465766963652059
:108E9C0028686578290000002045746865726E6545
:108EAC0074204D41432049442028686578296D354C
:108EBC002E6D342E6D332E6D322E6D312E6D30297C
:108ECC0000000000204761746577617920495020CB
:108EDC00286970332E6970322E6970312E697030AA
:108EEC0029200000204950206F6620746869732087
:108EFC0064657669636520286970332E6970322E3B
:108F0C006970312E697030290000000020537562A1
:108F1C006E6574204D61736B206F66207468697385
:108F2C002064657669636520286D332E6D322E6D55
:108F3C00312E6D3029000000204D756C7469636111
:108F4C00737420554450204D494449204D65726737
:108F5C0065204950286970332E6970322E69703142
:108F6C002E69703029000000204D49444928696E53
:108F7C00292D3E4D756C746963617374204465735F
:108F8C0074696E6174696F6E2854782920506F7201
:108F9C0074206E756D62657220284D657267652947
:108FAC0000000000204D756C746963617374204C73
:108FBC006F63616C285278292D3E4D494449286FC6
:108FCC0075742920506F7274206E756D62657220F5
:108FDC0028446973747269627574696F6E2F53706B
:108FEC006C69742900000000205374642E554450A1
:108FFC002F436F6D2044657374696E6174696F6E75
:10900C0020495020696E636C2E42726F61646361FB
:10901C007374286970332E6970322E6970312E6921
:10902C007030290020554450204C6F63616C2852DD
:10903C00782920506F7274206E756D6265722028CD
:10904C007374642E5544502C206E6F74204D756CC7
:10905C00746963617374290020554450204465730E
:10906C0074696E6174696F6E2854782920506F7220
:10907C0074206E756D62657200000000204C616E8C
:10908C00204D6F64653A20303D554450204D756C31
:10909C00746963617374204D657267652C20313D72
:1090AC007374642E554450204D657267652C2032C4
:1090BC003D5443502655445020434F4D0000000072
:1090CC002053706C69742F4469737472696275747F
:1090DC0065204D4944493420494E20746F204D4938
:1090EC004449312C332C35204F55543A20303D4EC9
:1090FC004F2C20313D594553000000002053706C1B
:10910C0069742F44697374726962757465204D4972
:10911C0044493520494E20746F204D494449312C27
:10912C00332C34204F55543A20303D4E4F2C2031A7
:10913C003D5945530000000020426974303A626C7E
:10914C006F636B2054696D696E67436C6B2C2042A6
:10915C006974313A626C6F636B2041637453656E52
:10916C00732C20426974323A626C6F636B205475B5
:10917C006E65526571000000204D49444931204F05
:10918C0055542046696C74657220666F7220434892
:10919C002E312D313620283420686578206E696296
:1091AC00626C65732058585858290000204D49446A
:1091BC004933204F55542046696C74657220666F94
:1091CC00722043482E312D313620283420686578A2
:1091DC00206E6962626C65732058585858290000DB
:1091EC00204D49444934204F55542046696C7465D0
:1091FC007220666F722043482E312D313620283470
:10920C0020686578206E6962626C657320585858C6
:10921C0058290000204D49444935204F55542046CB
:10922C00696C74657220666F722043482E312D3143
:10923C003620283420686578206E6962626C65730C
:10924C0020585858582900002045746865726E657E
:10925C0074204F55542046696C74657220666F7289
:10926C002043482E312D3136202834206865782053
:10927C006E6962626C65732058585858290000005A
:10928C0020555342204F55542046696C746572200A
:10929C00666F722043482E312D31362028342068D9
:1092AC006578206E6962626C65732058585858292D
:1092BC0000000000205443502F436F6D20506F72FC
:1092CC0074206E756D626572202854656C6E6574C1
:1092DC002F434F4D20706F7274206F6E6C792C2061
:1092EC006E6F7420666F72204D49444929202121EC
:1092FC00000000002054435020446973636F6E6E6D
:10930C006563742054696D65202830202E2E2E2024
:10931C003635353335207365636F6E64732C2030AE
:10932C003D6E6F206175746F20646973636F6E6E30
:10933C00656374290000000020434F4D34204261C6
:10934C00756472617465202855445026544350202E
:10935C00434F4D202B205365747570206F6E6C79C4
:10936C00293A2066697273742032206469676974C3
:10937C00732C4D4944493D333100000020434F4D7F
:10938C003420426175647261746520284D494449EA
:10939C00204D6572676572206F7065726174696FBC
:1093AC006E293A2066697273742032206469676989
:0C93BC0074732C4D4944493D33310000CE
:0893C80035020008AD010008A8
:0493D0008901000807
:1093D40000000000EC02002054030020BC03002025
:1093E4000000000000000000000000000000000079
:1093F4000000000000000000000000000000000069
:1094040000000000808D0008000000000000000043
:109414000000000000000000000000000000000048
:109424000000000000000000000000000000000038
:109434000000000000000000000000000000000028
:109444000000000000000000000000000000000018
:109454000000000000000000000000000000000008
:1094640000000000000000000000000000000000F8
:1094740000000000000000000100000000000000E7
:109484000E33CDAB34126DE6ECDE05000B000000AC
:1094940000000000000000000000000000000000C8
:1094A40000000000000000000000000000000000B8
:1094B40000000000000000000000000000000000A8
:1094C4000000000000000000000000000000000098
:1097F4000000000000000000F0880020CC1A0020C7
:10980400D09E0020785C002010730020B43000202B
:1098140098460020B0B40020206E6F55534221209A
:109824000000000000093D007C4E01206C64012012
:049834007876012021
:040000050800409D12
:00000001FF
